:10623A0001190000770101030200000301FA0400BA
:10624A00FA0500030A0A5A0B001E0C00FA0D000395
:10625A000E00040F0164100096120132130AFA1498
:10626A00020215000017010A1801FA1905321A016B
:10627A000A1B01FA1C05321FFFFF20FFFF23011E24
:10628A002400642A00FA2B00FA2C50782D003C2EA8
:10629A0000462F001E30006432507833000034323A
:1062AA00FA350164360164370150380A643C0064E7
:1062BA003E003C3F000040FFFF411450420A5A434F
:1062CA000AC84405324500B44600FA4701064802A6
:1062DA00034C00FA4EFFFF500606510596520A3249
:1062EA00530B46540A96560102570546580002595E
:1062FA000A465A32FA5B010A5C0A325E000A5F00F9
:10630A00FE61FFFF64FFFF66000267FFFF6A0A3C47
:10631A006B00006C329673000074000078013279C9
:10632A0001327EFFFF81FFFF84FFFF8500AF8600F9
:10633A00018700FA89010A8A00009900009D0A96DD
:10634A009E00019FFFFFA0FFFFFAFAFA0000770103
:10635A0001030200000301FA0400FA0500030A0A15
:10636A005A0B001E0C00FA0D00030E00040F016404
:10637A00100096120132130AFA14020215000017CD
:10638A00010A1801FA1905321A010A1B01FA1C0539
:10639A00321FFFFF20FFFF23011E2400642A00FA98
:1063AA002B00FA2C50782D003C2E00462F001E3070
:1063BA0000643250783300003432FA350164360111
:1063CA0064370150380A643C00643E003C3F0000D8
:1063DA0040FFFF411450420A5A430AC84405324555
:1063EA0000B44600FA4701034802024C00FA4EFF85
:1063FA00FF500606510596520A32530B46540A9626
:10640A00560101570546580001590A465A32FA5BA5
:10641A00010A5C0A325E000A5F00FE61FFFF64FF48
:10642A00FF66000267FFFF6A0A3C6B00006C329647
:10643A007300007400007801327901327EFFFF8117
:10644A00FFFF84FFFF85FFFF86FFFF87FFFF8901AC
:10645A00028A00009900009D0A969E00019FFFFF94
:10646A00A0FFFFFAFAFA0065006F00790083008D39
:10647A00009700A100AC00B600C000CA00D400DE3C
:10648A0000E800F2005800600068007000780080A0
:10649A0000880090009800A000A800B000B800C1D1
:1064AA0000C800D000D800DF00E600EE00F6004188
:1064BA000047004D00530059005F0065006C0071F1
:1064CA000077007D00830089008F0095009B00A261
:1064DA0000A700AC00B200B900C000C500CA00D2D3
:0A64EA0000D500DD00E100E700EF3F
:103A390090004CE0D3940440149007BDE0FEA3E04D
:103A4900FF90623C12662DE493F59980129007BDB0
:103A5900E0FEA3E0FF90635612662DE493F599907A
:103A690007BDE0FEA3E0FF90623AE493FC74019382
:103A7900FDEFB50507EEB50403754D009007BD12BE
:103A890066142275A71085F97385FA747E017F0083
:103A9900E574126606E5732FFF50010E8E5A8F5B8F
:103AA900900017E0FCA3E0FDEF2DFDEE3CFC8C5CE3
:103AB9008D5D2275A71085F97385FA747E017F00E3
:103AC900E574126606E5732FFF50010E8E5A8F5B5F
:103AD900AC2CAD2DEF2DFDEE3CFC8C5C8D5D22E513
:103AE9005DF5FBE55CF5FCD29322E55DF5E9E55C66
:103AF900F5EAD29422E55DF5EBE55CF5ECD291228D
:103B0900E55DF5EDE55CF5EED29222E55DF5FDE5C5
:103B19005CF5FED28722E55DF5CEE55CF5CFD29066
:103B290022AE5AAF5B74788E048F05FF1265F68C4E
:103B39005C8D5DAE5AAF5B74788E048F05FF12669B
:103B4900218C5A8D5BE55B455A60137478C3955B8C
:103B5900FFE4955AFE8E5A8F5B785C12665AE573BC
:103B6900A85CB80015D3955D4010E573C3955DFF5A
:103B7900E4955CFE8E5C8F5D8010E5732403C3952C
:103B89005DFFE4955CFE8E5C8F5D2290008DE0B454
:103B99000104C2128002D21290008EE0B40104C264
:103BA900138002D2139000CBE075F0DCA4FFAEF0D5
:103BB900740A8E048F05FF1265F69007B3ECF0A323
:103BC900EDF0A20D401674038C068D07126606747B
:103BD900011200399007B1EEF0A3EFF07E017F00EA
:103BE900900089E01266069000CCE08E048F05FFF4
:103BF9001265F6740AFF1265F68D609000D5E075BE
:103C0900F0DCA4FFAEF0740A8E048F05FF1265F68E
:103C19009007B7ECF0A3EDF09000D7E060139000A7
:103C2900D7E0F5F0741684FF7E00EF9007C5F080A9
:103C39000674649007C5F09000CDE0900071F09093
:103C49000117E090005BF09000A6E090005DF09015
:103C590000CFE090005EF090007BE090005FF09074
:103C69000101E0900064F0900165E0900065F0903A
:103C79000166E0900066F0900167E0900067F0A2AD
:103C89002CB34016900165E0700C900166E0700657
:103C9900900167E060028002C22C74E3900070F02A
:103CA9009000B6E0B40B0874E3900070F0805A906D
:103CB90000B6E0B419129000CCE090645B12008C5D
:103CC900E493900070F080419000B6E0B41E129029
:103CD90000CCE090647912008CE493900070F0803D
:103CE900289000B6E0B428129000CCE09064A312AA
:103CF900008CE493900070F0800F9000B6E0B44619
:103D0900089000ADE0900070F09000E6E0FE9000B1
:103D1900B4E06E600A9000B4E09000E6F0D22B9017
:103D29000074E0FE9000B3E0B50633900076E0FE43
:103D39009000D1E0B50627900075E0FE9000DFE025
:103D4900B5061B900078E0FE900086E0B5060F905E
:103D59000077E0FE9000C1E06E7003023F1890000A
:103D69004CE0C3940550087402900102F0801C9045
:103D790000C1E0640360069000DFE060087407900A
:103D89000102F08006740A900102F0900086E0B406
:103D9900010674009000ECF0900086E0B40206740D
:103DA900009000D1F0900086E0B403067400900002
:103DB900DEF09000B3E06014741890009AF074007B
:103DC9009006C7F074009006C8F0800C740090004B
:103DD9009AF074189006C7F09000D1E0D39401408E
:103DE900147419900104F074009006CBF0740090DB
:103DF90006CCF0800C7400900104F074199006CB85
:103E0900F09000C1E0B403089000DFE064026002B2
:103E1900800674009000DFF09000DFE0B4010890A4
:103E290000C1E064036002801A741A900105F074FD
:103E39000090009BF074009006CFF074009006D0BB
:103E4900F080339000B3E0B4021A741A90009BF02A
:103E59007400900105F074009006CFF0740090068C
:103E6900D0F08012740090009BF07400900105F06E
:103E7900741A9006CFF09000C1E0B402069000DFFA
:103E8900E06002801474049006DBF074059006DF8C
:103E9900F074069006E3F0802474009006DBF07459
:103EA900009006DCF074009006DFF074009006E0E4
:103EB900F074009006E3F074009006E4F0D22B90C1
:103EC90000B3E0900074F09000DFE0900075F0908E
:103ED90000D1E0900076F09000C1E0900077F0907A
:103EE9000086E0900078F0900086E090005CF09009
:103EF90000C1E0900060F09000DFE0900061F09078
:103F090000B3E0900062F09000D1E0900063F0907F
:103F190000E9E0B40117900023740FF0A374FFF0D7
:103F2900900025E4F0A3F074029000E9F09000E914
:103F3900E0B40341900025E0FEA3E0FF900023E0F8
:103F4900FCA3E0FD12665274101266067408120092
:103F590039EF90006DF0EF700674FF90006DF0740A
:103F6900009000E9F0900024E090006EF0900023AA
:103F7900E090006FF090007AE090003FF090003FF1
:103F8900E004900040F090003FE02402900041F0EE
:103F9900900040E0D39403400B900040E0C39403A9
:103FA900900040F0900041E0D39403400B90004111
:103FB900E0C39403900041F07551019000C0E09076
:103FC9000042F0900042E0D39403400F900042E099
:103FD900C39403900042F0D2258002C2259000428A
:103FE900E004900043F0900042E02402900044F085
:103FF900900043E0D39403400B900043E0C3940343
:10400900900043F0900044E0D39403400B900044A7
:10401900E0C39403900044F022C293C294C291C2B7
:1040290092C287C290E5B554EFF5B5E5B554DFF511
:10403900B5C296C295C2A0C297C2A2C2A1E5B554A3
:10404900BFF5B5E5B5547FF5B5E5B554FBF5B5C292
:1040590014755E469000C3E07005756D02800375A6
:104069006D0375550075540090000C74FFF0A3742E
:10407900DCF0C21AC21CC21E74C8900039F074C8A0
:1040890090003BF074C890003DF0755300755200E4
:10409900C20D754600E56FB40903756F00756300BD
:1040A900900019E4F0A3F0757010C217C218C21974
:1040B9009007B3E0FEA3E0FF7403126606740112D1
:1040C90000399007B1EEF0A3EFF0C2027557007501
:1040D9005600900010E4F0A3F0C22D7559007558F0
:1040E90000900085E075F032A4FDACF0900021EC61
:1040F900F0A3EDF09000377475F0A37430F0C20EA0
:10410900C20FC23DA231B39205A232B39206A233C5
:10411900B39207A234B39208A235B39209A236B377
:10412900920AA237B3920BA238B3920C2275A71048
:1041390085F97385FA747E017F00E574126606E5D8
:10414900732FFF50010E8E5A8F5BAC5CAD5DEF2D66
:10415900FDEE3CFC8C5C8D5D123AE8123AF3123AA2
:10416900FE9000C1E0B40309123B09123B14123B53
:104179001F75A7002285F97385FA747E017F00E512
:1041890074126606E5732FFF50010E8E5A8F5B7EFF
:10419900017F769000FEE0126606AC5AAD5BED2F0A
:1041A900FFEC3EFE8E5C8F5DE55DF5EDE55CF5EEC1
:1041B900900071E4F07412900048F02285F973853B
:1041C900FA747E017F00E574126606E5732FFF50CD
:1041D900010E8E5A8F5B9007B3E0FCA3E0FDEF2D33
:1041E900FDEE3CFC8C5C8D5DE55DF5FDE55CF5FE69
:1041F90022056422A2DBB340089000CDE090007153
:10420900F0A2DCB34006C296C295C2A075D840227E
:1042190085A77275A7109000C1E06403600790003C
:10422900DFE0B4022CA2D8B34002C293A2D9B340B2
:1042390002C294A2DAB34002C291A2DBB34002C225
:1042490092A2DCB34002C287A2DDB34002C29080D1
:104259002DA2D8B3400AC2939000DFE06002C29257
:10426900A2D9B3400AC2949000DFE06002C287A2DB
:10427900DAB3400AC2919000DFE06002C29075D8BB
:10428900408572A722900047E4936406600280FE8D
:1042990074C89007B9F8E4F0E8A3F075B50075841F
:1042A9000175A70075FFA0900045E4F075C9107568
:1042B900A70F75A1C775A70075D90075CE0C75A78D
:1042C9000F75F1FE75F2FF75F30775F47875A4BAE9
:1042D90075A5FF75A60775AE0075AFFF75D4817515
:1042E900D5FF75D6FF75D7FF75A70075A20175A112
:1042F9004775F80975D80075D90475DD0975DE09A2
:1043090075D84075A71075D80075D90475DA09757F
:10431900DB0975DC0975DD0975DE0975DF0975D8F5
:104329004075A70075E60875E71075BC0175BE04F0
:1043390075BD6C75BE0775BDA075BE0875BD0175E7
:10434900BC0075BB1875BC2075BA0875E88075D1B5
:104359001375A70F75E10575E20075C74012402274
:10436900759700759780740A1265E67597C0E59789
:104379005420700280F8758F0275A700D2AF759826
:104389000075A90C75A70F75AB4375ADFB75AC1E10
:1043990075A71075C91875CA0075CB0075C804755D
:1043A900A700758912758E04758C00758A00C2A9DB
:1043B900D28C758D00758B00D2ABD28E75EF0675D8
:1043C900D944C29974C8F5097508001200E975B590
:1043D900001204E974639007B9F8E4F0E8A3F01255
:1043E900037574C89007B9F8E4F0E8A3F07464F5AC
:1043F900097508001200E990005CE0900086F090D1
:104409000086E0D39403400C7400900086F0740099
:1044190090005CF0C222900086E0905E4BF828285C
:10442900738028A2B44002D222802075A70F75F3A9
:104439000F75A700A2A34002D222800F75A70F759E
:0B444900F31775A700A2A44002D222C6
:0C5E4B0002442A02442C02443402444564
:10445400A222B3405F757308E573D3940E5020E530
:10446400739007B9F8E4F0E8A3F01202447464F519
:10447400097508001200E97873740126F650D9749E
:10448400029000C2F090005CE0900086F0900086FC
:10449400E0905E57F8282873801674009000ECF0C2
:1044A400800E74009000D1F0800674009000DEF05D
:0C5E570002449C02449E0244A60244AE99
:1044B400D221805D757301E573D394075020E573B1
:1044C4009007B9F8E4F0E8A3F01202447464F50923
:1044D4007508001200E97873740126F650D9740146
:1044E4009000C2F090005CE0900086F0900086E0BE
:1044F400905E63F8282873801674009000ECF080B6
:0F4504000E74009000D1F0800674009000DEF07D
:0C5E63000244FB0244FD02450502450D0F
:10451300C22190005BE0900117F090005CE09000F6
:1045230086F090005DE09000A6F090005EE09000C1
:10453300CFF090005FE090007BF0900060E090008F
:10454300C1F0900061E09000DFF0900062E0900025
:10455300B3F0900063E09000D1F0900064E090012C
:1045630001F0900065E0900165F0900066E0900135
:1045730066F0900067E0900167F0900165E0700CD1
:10458300900166E07006900167E060028004C22C2F
:104593008002D22C9000CCE07006740A9000CCF01C
:1045A3009000ADE0700674E39000ADF09000B3E0CE
:1045B30004900074F09000B4E09000E6F0123B9495
:1045C300E5B54401F5B5740690004AF07401900016
:1045D3004BF0740390004DF0740590004EF0742876
:1045E30090004FF07405900050F090004CE0B4043C
:1045F300067404900050F07401900051F074009020
:104603000056F07400900059F074FF90005AF07453
:104613004E900150F07469900151F07473900152FF
:10462300F07473900153F07461900154F0746E90C0
:104633000155F07420900156F07436900157F074D0
:1046430043900158F07479900159F0746C90015AB9
:10465300F0742090015BF0742090015CF074209062
:10466300015DF0742090015EF09000E8E090006D31
:10467300F090009FE090006EF09000A0E090006F3B
:10468300F0A2B6B39210A2B3B39211A2A4B392282C
:10469300A2B4B39229A2A3B3922A900069E4F0755D
:1046A3006F00743A900779F074FD90077AF09000E8
:1046B3006AE4F09007B3E0FEA3E0FF74031266061A
:1046C30074011200399007B1EEF0A3EFF0756E019B
:1046D300900048E4F0C227756300C215D216C202E7
:1046E300757100C22FD203C230D204C231D205C2C7
:1046F30032D206C233D207C234D208C235D209C27B
:1047030036D20AC237D20BC238D20CC223C224C259
:1047130025C226C22B12009E755F00756B00756162
:104723000075653275660075670075680075690008
:10473300756A00900019E4F0A3F0756C00D2B2D250
:10474300A4D2B0D2B1D2A3D2A7D2A6D2A5D2B790C7
:104753000085E0D394FA400674FA900085F07E0158
:104763007F0090006FE012660690006EE02FFF500E
:10477300010E900023EEF0A3EFF0EFD394FFEE943D
:104783000F4007900023E4F0A3F090006DE0700663
:1047930074FF90006DF09000C2E0D3940240067461
:1047A300019000C2F09000C3E07005756D028003B4
:1047B300756D039000C4E0D394014006740090002B
:1047C300C4F09000CAE0C3940A5006740A9000CA69
:1047D300F09000D4E0700674019000D4F09000D4FF
:1047E300E0B4FF0674FE9000D4F09000DBE0D394B5
:1047F300FE400674FE9000DBF0900101E0D39402CA
:1048030040067401900101F0900117E0D394014038
:10481300067401900117F074019000E1F0740190A7
:1048230000E2F074009000E9F07400900109F07464
:10483300299006BFF0742A9006C3F0741B9006D328
:10484300F0741C9006D7F0D29C9000B4E0D394048B
:10485300400674049000B4F0E570D39410400375DF
:1048630070109006C0E0D3940C400674009006C00C
:10487300F09006C4E0D3940C400674009006C4F094
:104883009006C8E0D3940C400674009006C8F090DC
:1048930006CCE0D3940C400674009006CCF090064E
:1048A300D0E0D3940C400674009006D0F09006D468
:1048B300E0D3940C400674009006D4F09006D8E040
:1048C300D3940C400674009006D8F09006DCE0D335
:1048D300940C400674009006DCF09006E0E0D3945C
:1048E3000C400674009006E0F09006E4E0D3940CCC
:1048F300400674009006E4F0D2EC75CF01A298B3A1
:104903004005C298120646E54D6006A299B3B3402E
:10491300028005C299120C57E54E64016005E54E0D
:10492300B4040280D5C28E7E107F00E56412660651
:10493300E58D75F010A4FDACF0EF2DFDEE3CFCE52C
:104943008B75F01084FF7E00ED2FFFEC3EFE8E543E
:104953008F55D28E9000A6E0605690001B1266140D
:1049630090001BE0FCA3E0FD90001DE0FAA3E0FB38
:10497300EDB5033CECB50238B220A20DB34013A24F
:1049830020B34008E5B54404F5B58006E5B554FB0E
:10499300F5B590001DE0FEA3E0FF90001FE0FCA32F
:1049A300E0FDEF2DFDEE3CFC90001DECF0A3EDF0DF
:1049B3009000B3E060099000B3E0C3940340028029
:1049C3006F122D96A20DB35009900069E0C3940BAA
:1049D3004002800690009DE0F545E54575F005A48D
:1049E300FFAEF09007BBEEF0A3EFF090008AE0C3B8
:1049F30095614007E55FC3956050079007BBE4F0FE
:104A0300A3F0AE2EAF2F9007BBE0FCA3E0FDEFD3E6
:104A13009DEE9C4004C297800B900069E0C3941103
:104A23005002D2979000B3E0B40205A297B392A1CB
:104A33009000B3E0B4031C122EB1AE2EAF2F90073B
:104A4300BBE0FCA3E0FDEFD39DEE9C4004D2978036
:104A530002C297A2B6301001B35003024FB1A2B6FF
:104A6300301001B35003024FB1A2B6301201B3505C
:104A730003024DE1756E00055EA20EB35003024BB7
:104A830035E56DB4032EA22DB34022E55EB40703D2
:104A9300756D01E55EC3940750069000487401F0FC
:104AA300E55ED3940740067402900048F0755E01FA
:104AB300D22D805AE56DB40206756D01755E04E56D
:104AC3005EB40405755E018045900048E07030E5F2
:104AD3005EC3940450069000487401F0E55ED394DD
:104AE3000440067402900048F0E55EC3940450024B
:104AF300D227E55ED394044002D227C296C2959092
:104B030000C3E0B401051240228003755E01C20EAA
:104B1300C20FA2259224A2B4B34002C229A2A4B315
:104B23004002C228A2A3B34002C22AA227B3400272
:104B3300C227E56DC394035006E55E6404600280FA
:104B430016B224755E01A20F4004B20F80097405EA
:104B5300900048F01240229000C1E0B40308900096
:104B630042E0655E6002800BA224B34004D226803B
:104B730002C226E55EB403499000A6E060439000BC
:104B83001BE0FEA3E0FF9000A6E08E048F05FF125A
:104B930065F674018C068D0712003990001FEEF044
:104BA300A3EFF090001FE0F8A3E090001DC8F0A36E
:104BB300C8F090001BE4F0A3F0C220E5B554FBF568
:104BC300B5AE58AF59AC54AD55EF2DFDEE3CFC8C52
:104BD300588D59AE54AF55EFD39DEE9C40119000C4
:104BE30013E0FAA3E0FBEBC394E8EA9403400280EA
:104BF3000690001312661490000CE554F0A3E555DB
:104C0300F090000EE554F0A3E555F0AE54AF5574A3
:104C13000C8E048F05FF1265F68C568D57C28E7568
:104C23008D00758B00756400755501755400D28E27
:104C330090000CE0FEA3E0FFEF4E600B7CAC7D60C8
:104C43001264F48E528F53AE52AF537428BE0003D6
:104C53009F5010E5632FFF50010E74011200398E2F
:104C6300528F538553639000CAE0A852B8000DD306
:104C730095534008E553900047F080099000CAE03F
:104C830014900047F0E56D6006755300755200E51A
:104C93005E64016005E55EB403099000B3E0600360
:104CA3001223D2E56FB40903756F00A215500302F6
:104CB3004D5A90007FE0B40173900101E0B40214F7
:104CC300120E26900072E075F0BEA4FFAEF08E5C6B
:104CD3008F5D8056E56775F00A84FF7E0090057945
:104CE30012662DE0F55B755A00AE5AAF5B9000A4D7
:104CF300E012660674648E048F05FF1265F68C5C01
:104D03008D5DE55D900012F0AE5AAF5B90007DE0E3
:104D130012660674648E048F05FF1265F674BE8CEA
:104D2300068D071266068E5C8F5D801790007DE00E
:104D330075F0BEA4FFAEF08E5C8F5D9000A4E09092
:104D43000012F0E561C394CC5006E55D455C70024A
:104D53008003124136D215E56DB40106A214B3B334
:104D6300400280097570019000497401F0E56D708F
:104D7300689000C6E0600D900071E0A852B800068C
:104D83009553400280299000C6E0B4020875700371
:104D9300756C00800CC200756C00900019E4F0A3E0
:104DA300F0900071E060067409900048F0802A7565
:104DB300700190003FE0B55E069000497401F090E9
:104DC3000040E0B55E067402900049F0900041E0B7
:104DD300B55E067403900049F0A212B39210A212BA
:104DE300B330B601B35003024FB1756E01E5B5445C
:104DF30001F5B5740B900069F0A2129210E55ED331
:104E030094484014D214E55ED3944E400B7405903D
:104E13000048F0D227755E469000CEE0B40107E566
:104E23006AC394144002800912402274139000480C
:104E3300F0A214B3B35018900037E0FEA3E0FF7460
:104E430002126606AC54AD55EFC39DEE9C40028042
:104E530002D20E900037E554F0A3E555F0A22F30AF
:104E63000301B35017A22FB34008E5B54408F5B5C5
:104E73008006E5B554F7F5B5A22F9203A2303004AE
:104E830001B35017A230B34008E5B54402F5B5802D
:104E930006E5B554FDF5B5A2309204A23130050103
:104EA300B3500FA231B34004D2978002C297A2310C
:104EB3009205A232300601B3500FA232B34004D29E
:104EC300A28002C2A2A2329206A233300701B350DB
:104ED3000FA233B34004D2A18002C2A1A23392072E
:104EE300A234300801B35017A234B34008E5B544E7
:104EF30040F5B58006E5B554BFF5B5A2349208A2D6
:104F030035300901B35017A235B34008E5B54480E5
:104F1300F5B58006E5B5547FF5B5A2359209A236FD
:104F2300300A01B3500FA236B34004D2928002C2BA
:104F330092A236920AA237300B01B3500FA237B3B5
:104F43004004D2878002C287A237920BA238300C6A
:104F530001B3500FA238B34004D2908002C290A292
:104F630038920CE56AC394415009740E900048F0DE
:104F7300124022900050E0FE90004CE004C39E409B
:104F83000990004CE0D39408400974FB900048F06A
:104F9300124022900055E06015900055E0FE90000D
:104FA3004FE06E600974FE900048F0124022A22781
:104FB300B34006C296C295C2A09000FEE0600CAE5C
:104FC30052AF537414BE00059F4002804890008680
:104FD300E0905E6FF8282873803BA2B4B35005A21B
:104FE30029B34002800512417ED2298028A2A3B3AF
:104FF3005005A22AB34002800512417ED22A8015B1
:10500300A2A4B35005A228B34002800512417ED268
:0550130028800280006E
:105E6F00024FDB024FDD024FF002500302501602C9
:025E7F005018B9
:10501800A217B3B35008900042E0655E60030250E7
:10502800ADA201B35006A200B3B340028071900054
:10503800C1E0B40343123A8CA20DB34021A226B3B7
:105048004005123AE88003123B099000DFE0B40102
:105058000BA202B34004D2A18002C2A18018123A66
:10506800E8123B099000DFE0B4010BA202B3400450
:10507800D2A18002C2A180249000DFE0C394025034
:105088000F123A8C123AE8A202B34002D292800C74
:10509800123A8C123AE8123ABC123B0975A700C2C0
:1050A80017D218D219A218B3B35008900043E0657C
:1050B8005E6003025142A201B35006A200B3B3409E
:1050C8000280719000C1E0B40343123A8CA20DB380
:1050D8004021A226B34005123AF38003123B1490F4
:1050E80000DFE0B4010BA202B34004D2A18002C2E7
:1050F800A18018123AF3123B149000DFE0B4010BC0
:10510800A202B34004D2A18002C2A180249000DF91
:10511800E0C39402500F123A8C123AF3A202B34041
:1051280002D287800C123A8C123AF3123ABC123B24
:105138001475A700D217C218D219A219B3B3500810
:10514800900044E0655E60030251D7A201B35006A7
:10515800A200B3B3400280719000C1E0B4034312CF
:105168003A8CA20DB34021A226B34005123AFE8024
:1051780003123B1F9000DFE0B4010BA202B340040E
:10518800D2A18002C2A18018123AFE123B1F9000E1
:10519800DFE0B4010BA202B34004D2A18002C2A195
:1051A80080249000DFE0C39402500F123A8C123A28
:1051B800FEA202B34002D290800C123A8C123AFE40
:1051C800123ABC123B1F75A700D217D218C219E5B4
:0F51D80070905E81F82828730256189000B4E09A
:065E81000251E00251E3B2
:1051E700905EB4F8282873121EAE8012121EAE808D
:0E51F7000D121F388008121FE48003121FE4FF
:0F5EB4000251EE0251F30251F80251FD02520267
:10520500757002025618122110122227A23DB340D2
:105215000C9000A8E0F56C7410900048F0900079AF
:10522500E0256CF5369007B1E0FEA3E0FF7414129B
:10523500660690000EE0FCA3E0FD74068F02FF12E7
:1052450065F68D078C038E048A058B061264F4902F
:1052550007B5EEF0A3EFF09000CFE0B40108744677
:10526500BE00059F4002800D74469007B5F8E4F036
:10527500E8A3F0801B9007B5E0FEA3E0FF74F0BE45
:1052850000039F500B74F09007B5F8E4F0E8A3F025
:10529500E53670037536019007B5E0FEA3E0FFE53E
:1052A500362FFF50010E9007B5EEF0A3EFF07570A5
:0552B50003900049E038
:035E870002520BB9
:1052BA00905EC3F82828738019A23E400375700ACD
:1052CA008010A23E400375700B8007A23E40037512
:0252DA00700C56
:0C5EC3000252C10252C30252CC0252D55E
:1052DC000256189006C0E060031224EA9000FFE02A
:1052EC00B40114900100E0A852B800049553500783
:1052FC00E55FC39560400280097415900048F00288
:10530C00538F9000B4E0D39402403F900088E02487
:10531C0003A852B800049553500990008AE0D39525
:10532C006150028008D2017408900048F090008807
:10533C00E0A852B80005D39553500B90008AE02496
:10534C0003C395615002C2018039900088E02403A8
:10535C00A852B8000495535007E55FC3956040020E
:10536C008008D2017408900048F0900088E0A852A0
:10537C00B80005D395535009E560240FC3955F50D1
:10538C0002C2019000CEE07007E56AC3941440029B
:10539C008002D201A2014005757004800A7570105C
:1053AC00900019E4F0A3F0A20DB34029E56775F065
:1053BC000A84FF7E0090057912662DE0C394695033
:1053CC0005122407800F9007B3E0F8A3E09007B113
:0C53DC00C8F0A3C8F00256189000B4E01E
:065E8A000252DF0253E4A6
:1053E800905ECFF8282873120F108012120F1080C9
:0E53F8000D1210BE8008121170800312117089
:0F5ECF000253EF0253F40253F90253FE0254033D
:105406009006C4E060031225C67570050256181290
:1054160012B07570069006C8E060031226B69006B4
:10542600CCE06003122792025618900012E0600644
:10543600A20DB3B34002801D900012E02529FFAEF5
:105446002850010E8E288F29E55ED39401500690D0
:105456000012E014F01214F67570079006D0E060A2
:105466000312286E9006D4E0600312294A025618E9
:10547600900101E0B40203120E9E1218F575700831
:105486009006D8E06003122A269006DCE06003123C
:105496002B02025618121CB1A217B35005A218B35C
:1054A60040028006D217D218D2197570109006E005
:1054B600E06003122BDE9006E4E06003122CBA02D1
:1054C600561802561890003AE0C394465008C29601
:1054D600744690003AF085365B755A0090003FE0BE
:1054E600F573123B2AE55D90003AF0900006E55A06
:1054F600F0A3E55BF0C21B9007B5E0F55AA3E0F513
:105506005B90003FE0F573123B2AE55D900039F0B1
:10551600900000E55AF0A3E55BF0C21AE56DB40110
:105526000575700B800375700302561890003CE0F9
:10553600C3944650139000CFE0B40104C296800293
:10554600C295744690003CF085365B755A00900013
:1055560040E0F573123B2AE55D90003CF0900008B0
:10556600E55AF0A3E55BF0C21D9007B5E0F55AA336
:10557600E0F55B900040E0F573123B2AE55D900094
:105586003BF0900002E55AF0A3E55BF0C21CE56D26
:10559600B4010575700C8003757003807590003E2C
:1055A600E0C3944650139000CFE0B40104C2968045
:1055B60002C2A0744690003EF085365B755A009094
:1055C6000041E0F573123B2AE55D90003EF0900045
:1055D6000AE55AF0A3E55BF0C21F9007B5E0F55A5D
:1055E600A3E0F55B900041E0F573123B2AE55D9080
:1055F600003DF0900004E55AF0A3E55BF0C21EE51D
:105606006DB40103756D0075700380068004800219
:02561600800012
:105E900002541502543002547602549B0254C80234
:105EA00054CB0255320255A3025612025614025622
:045EB0001602561868
:10561800900039E0B55E0280030256B3A21A406BCF
:10562800900000E0FEA3E0FFEF4E605DAC52AD538A
:10563800740ABC0033D39D402FAA56AB5774058A11
:10564800048B05FF1265F68D068C07900000E0FCC0
:10565800A3E0FDCFCECF12000374011200399000F1
:1056680000EEF0A3EFF08021AE56AF57900000E0B7
:10567800FCA3E0FD120003740A8E048F05FF126577
:10568800F6900000ECF0A3EDF0D21AAE54AF5590AE
:105698000000E0FCA3E0FDEFC39DEE9C400D12412D
:1056A800C5D296C21A74C8900039F0A21AB3B35082
:1056B80007900039E0B55E02800D1241C5D296749C
:1056C800C8900039F0C21A90003AE0B55E02800333
:1056D800025767A21B406B900006E0FEA3E0FFEFB5
:1056E8004E605DAC52AD53740ABC0033D39D402F5D
:1056F800AA56AB5774058A048B05FF1265F68D060A
:105708008C07900006E0FCA3E0FDCFCECF1200038B
:105718007401120039900006EEF0A3EFF08021AE7C
:1057280056AF57900006E0FCA3E0FD120003740A90
:105738008E048F05FF1265F6900006ECF0A3EDF0DD
:10574800D21BAE54AF55900006E0FCA3E0FDEFC3BA
:105758009DEE9C400AC296744690003AF0C21BA285
:105768001BB3B3500790003AE0B55E02800AC296B8
:10577800744690003AF0C21B90003BE0B55E028090
:1057880003025826A21C406B900002E0FEA3E0FF33
:10579800EF4E605DAC52AD53740ABC0033D39D40EC
:1057A8002FAA56AB5774058A048B05FF1265F68D30
:1057B800068C07900002E0FCA3E0FDCFCECF1200DC
:1057C800037401120039900002EEF0A3EFF080217B
:1057D800AE56AF57900002E0FCA3E0FD1200037440
:1057E8000A8E048F05FF1265F6900002ECF0A3ED17
:1057F800F0D21CAE54AF55900002E0FCA3E0FDEFE0
:10580800C39DEE9C40181241C59000CFE0B401043E
:10581800D2968002D295C21C74C890003BF0A21C9C
:10582800B3B3500790003BE0B55E0280181241C543
:105838009000CFE0B40104D2968002D29574C8904B
:10584800003BF0C21C90003CE0B55E0280030258A9
:10585800F0A21D406B900008E0FEA3E0FFEF4E6051
:105868005DAC52AD53740ABC0033D39D402FAA5689
:10587800AB5774058A048B05FF1265F68D068C07F5
:10588800900008E0FCA3E0FDCFCECF120003740126
:10589800120039900008EEF0A3EFF08021AE56AF69
:1058A80057900008E0FCA3E0FD120003740A8E0480
:1058B8008F05FF1265F6900008ECF0A3EDF0D21DFD
:1058C800AE54AF55900008E0FCA3E0FDEFC39DEE99
:1058D8009C40159000CFE0B40104C2968002C295A6
:1058E800744690003CF0C21DA21DB3B3500790004F
:1058F8003CE0B55E0280159000CFE0B40104C2968A
:105908008002C295744690003CF0C21D90003DE0B4
:10591800B55E0280030259BAA21E406B900004E0F3
:10592800FEA3E0FFEF4E605DAC52AD53740ABC00BD
:1059380033D39D402FAA56AB5774058A048B05FFB5
:105948001265F68D068C07900004E0FCA3E0FDCFFD
:10595800CECF1200037401120039900004EEF0A3B8
:10596800EFF08021AE56AF57900004E0FCA3E0FDB5
:10597800120003740A8E048F05FF1265F690000466
:10598800ECF0A3EDF0D21EAE54AF55900004E0FC4D
:10599800A3E0FDEFC39DEE9C40181241C59000CFD7
:1059A800E0B40104D2968002D2A0C21E74C890004E
:1059B8003DF0A21EB3B3500790003DE0B55E0280F3
:1059C800181241C59000CFE0B40104D2968002D2EB
:1059D800A074C890003DF0C21E90003EE0B55E0283
:1059E8008003025A84A21F406B90000AE0FEA3E0E5
:1059F800FFEF4E605DAC52AD53740ABC0033D39DCB
:105A0800402FAA56AB5774058A048B05FF1265F61A
:105A18008D068C0790000AE0FCA3E0FDCFCECF12E4
:105A28000003740112003990000AEEF0A3EFF08031
:105A380021AE56AF5790000AE0FCA3E0FD12000328
:105A4800740A8E048F05FF1265F690000AECF0A325
:105A5800EDF0D21FAE54AF5590000AE0FCA3E0FD74
:105A6800EFC39DEE9C40159000CFE0B40104C296B0
:105A78008002C2A0744690003EF0C21FA21FB3B3BA
:105A8800500790003EE0B55E0280159000CFE0B46C
:105A98000104C2968002C2A0744690003EF0C21F64
:105AA8009000D1E0B402028003025BC490006BE076
:105AB800D39566506490006BE0F4042566FE900070
:105AC800D4E08E00F5F0E884FF7E008F73EFC39476
:105AD80010500CEF8573F0A4FDACF08D7380037546
:105AE80073FF90006BE0D39573400B90006BE0C39D
:105AF8009573F57180037571009000EFE0D395718F
:105B080040069000EFE0F5719000F0E0C395715009
:105B1800069000F0E0F571807190006BE0C3956627
:105B2800FE9000D4E08E00F5F0E884FF7E008F73CD
:105B3800EFC39410500CEF8573F0A4FDACF08D7397
:105B480080037573FF85735B755A0090006BE025C1
:105B58005BFFAE5A50010E8E5A8F5B74FFBE000970
:105B6800D39F4005855B7180037571FF9000EFE05E
:105B7800D3957140069000EFE0F5719000F0E0C316
:105B8800957150069000F0E0F571A20DB3B3500D79
:105B980090006CE0FE9000DCE0D39E5002800A7416
:105BA80007900048F0C2A2801375A710E5CDC395F1
:105BB800714004C2A28002D2A275A700E56FC39407
:105BC80009500AA2EDB34005C2ED123050AE54AFF1
:105BD800557450C39F74C39E400C90006AE0C394F0
:105BE8005A4003025E48A214B340091240227406C8
:105BF800900048F0A222B34008E5B54404F5B5800A
:105C080006E5B554FBF5B5A216B3500EE561D3947D
:105C1800334007E561C394CC40028041900101E024
:105C2800B40214120E26900072E075F050A4FFAE74
:105C3800F08E5C8F5D800F90007DE075F050A4FFC2
:105C4800AEF08E5C8F5DE55D455C6011E5B54401A5
:105C5800F5B5740B900069F0124136D21690006ABF
:105C6800E0D394014007E561C3941A40028002C260
:105C7800169006C0E060031224EAA22F300301B395
:105C88005017A22FB34008E5B54408F5B58006E5DE
:105C9800B554F7F5B5A22F92039006C4E06003123D
:105CA80025C6A230300401B35017A230B34008E52E
:105CB800B54402F5B58006E5B554FDF5B5A23092B8
:105CC800049006C8E060031226B6A231300501B37D
:105CD800500FA231B34004D2978002C297A23192EA
:105CE800059006CCE06003122792A232300601B379
:105CF800500FA232B34004D2A28002C2A2A23292B2
:105D0800069006D0E0600312286EA233300701B374
:105D1800500FA233B34004D2A18002C2A1A2339291
:105D2800079006D4E0600312294AA234300801B370
:105D38005017A234B34008E5B54440F5B58006E5F0
:105D4800B554BFF5B5A23492089006D8E0600312A6
:105D58002A26A235300901B35017A235B34008E509
:105D6800B54480F5B58006E5B5547FF5B5A2359202
:105D7800099006DCE06003122B02A236300A01B358
:105D8800500FA236B34004D2928002C292A2369239
:105D98000A9006E0E06003122BDEA237300B01B355
:105DA800500FA237B34004D2878002C287A237922D
:105DB8000B9006E4E06003122CBAA238300C01B351
:105DC800500FA238B34004D2908002C290A23892F9
:105DD8000C90006AE0C3945A5010E56FB40909901A
:105DE800006AE004F0756F00803BE56FB409037545
:105DF8006F00755500755400758D00758B007564BE
:105E080000900069E0C394115008900069E004F024
:105E180080067411900069F0900069E0B41106E5FD
:105E2800B554FEF5B590006AE0D394014007E56AE1
:105E3800C3944140028009740E900048F012402239
:035E48000248FD10
:105EDE000000010001400160018001A001C001E04D
:105EEE0002000300039603B603D603F40400050074
:105EFE000512052405360548055A056C057E0590E4
:105F0E0005A805C005DE0600061406280646066E20
:105F1E0006AE05CF00FF013F015F017F019F01BF6C
:105F2E0001DF01FF02FF039503B503D503F303FF62
:105F3E0004FF05110523053505470559056B057D3C
:105F4E00058F05A705BF05CE05F1061306270645E5
:105F5E00066D06AD06ED05DD0FAA0FA50F9F0F9A74
:105F6E000F940F8D0F870F800F780F710F680F60D2
:105F7E000F570F4E0F450F3B0F300F250F1A0F0EF9
:105F8E000F020EF50EE80EDB0ECC0EBE0EAE0E9F01
:105F9E000E8E0E7D0E6C0E5A0E470E340E200E0C0B
:105FAE000DF70DE20DCB0DB50D9D0D850D6D0D543F
:105FBE000D3A0D200D050CE90CCE0CB10C940C769F
:105FCE000C580C3A0C1B0BFB0BDB0BBB0B9A0B7917
:105FDE000B570B350B130AF10ACE0AAB0A870A646C
:105FEE000A400A1C09F809D409B0098C096709434B
:105FFE00091F08FB08D608B2088E086A084608234F
:10600E0007FF07DC07B9079607730751072F070D20
:10601E0006EC06CA06AA068906690649062A060A73
:10602E0005EC05CD05B0059205750558053C052016
:10603E00050504EA04CF04B5049C048204690451E6
:10604E0004390422040B03F403DE03C803B2039DD8
:10605E00038903750361034D033B032803160304F1
:10606E0002F202E102D102C002B002A0029102824B
:10607E000273026502570249023C022F02220216E7
:10608E00020901FD01F201E601DB01D001C601BBEF
:10609E0001B101A7019D0194018B0182017901706B
:1060AE000168016001580150014801410139013276
:1060BE00012B0125011E01180111010B010500FF25
:1060CE0000FA0FA60FA00F990F920F8B0F840F7C63
:1060DE000F740F6B0F620F580F4E0F430F380F2CAC
:1060EE000F1F0F120F050EF70EE80ED80EC80EB7C3
:1060FE000EA50E930E800E6C0E580E420E2C0E1523
:10610E000DFD0DE40DCB0DB10D950D790D5D0D3F12
:10611E000D200D010CE10CC00C9E0C7C0C590C35A5
:10612E000C100BEA0BC40B9E0B760B4F0B260AFDC5
:10613E000AD40AAA0A800A550A2A09FF09D409A80C
:10614E00097C0950092508F908CD08A10875084AE7
:10615E00081E07F307C8079D07730749072006F7B0
:10616E0006CE06A6067E06570630060A05E405BFCD
:10617E00059B057705540532051004EF04CE04AED9
:10618E00048F047104530435041903FD03E203C79D
:10619E0003AD0394037B0363034B0334031E030815
:1061AE0002F302DE02CA02B602A30291027F026D60
:1061BE00025C024C023C022C021D020E020001F295
:1061CE0001E401D701CA01BE01B101A6019A018FF6
:1061DE000185017A01700166015D0153014A014199
:1061EE00013901310129012101190112010B0104AB
:1061FE0000FD00F700F000EA00E400DE00D900D355
:10620E0000CE00C900C400BF00BA00B500B100AD99
:10621E0000A800A400A0009C009900950091008E9B
:0C622E00008A008700840081007E007B55
:10009E007547009007BDE4F0A3F075310075300090
:1000AE00754D00754E00C23AD23B74FE9007BFF8F4
:1000BE00E4F0E8A3F074FE9007C1F8E4F0E8A3F0D2
:1000CE0074FE9007CBF0745A9007CCF0745A9007D8
:1000DE00CDF0D23CC22EC23EC23922750B00750A3B
:1000EE0000AE0AAF0BAC08AD09EDC39FEC9E4016F7
:1000FE0074FF1265E675CF01780B740126F6500475
:10010E0018E436F650DB22900045E0B4AA1C9007A6
:10011E0079E0B43C159007B9E0FEA3E0FFEF4E6026
:10012E0009741EBE0004D39F5003020243755D0086
:10013E00755C0075F8099007B9E0FEA3E0FF74073F
:10014E006F4E6006740E6F4E7006743A900779F01B
:10015E009007B9E0FEA3E0FF7408BE001ED39F40D7
:10016E001A7E017F089007B9E0FCA3E0FD1DBDFFDC
:10017E00011C1200038E5A8F5B801F9007B9E0FEA0
:10018E00A3E0FF740812664A8F048E057E017F0875
:10019E00CDCCCD1200038E5A8F5BAE5CAF5D740C6E
:1001AE00D39F74019E500302023EA2F9B3407EE536
:1001BE005D455C700375A382AE5CAF5D74016F4EDE
:1001CE00700375A300AE5CAF5D74026F4E700D9040
:1001DE0007BAE075F002A4FDACF08DA3AE5CAF5D86
:1001EE0074036F4E700375A300AE5CAF5D7403BEF7
:1001FE0000039F5013AC5AAD5BED2FFFEC3EFE900B
:10020E00007512662DE0F5A3AE5CAF5DEFB40B0981
:10021E00EEB4010574141265E6AE5CAF5DEFB40B7F
:10022E0007EEB4010375F80D785C12665A0201A848
:10023E00900045E4F022755D00755C0075F809903C
:10024E0007B9E0FEA3E0FF7408BE001ED39F401A5C
:10025E007E017F089007B9E0FCA3E0FD1DBDFF0104
:10026E001C1200038E5A8F5B801F9007B9E0FEA30D
:10027E00E0FF740812664A8F048E057E017F08CD5A
:10028E00CCCD1200038E5A8F5BAE5CAF5D7411D372
:10029E009F74019E5003020374A2F9B3500302032C
:1002AE0071E55D455C700375A3D2AE5CAF5D740104
:1002BE006F4E700375A300AE5CAF5D74026F4E702F
:1002CE000D9007BAE075F002A4FDACF08DA3AE5C04
:1002DE00AF5D74036F4E700375A300AE5CAF5D74BB
:1002EE00046F4E700375A300AE5CAF5D74056F4E68
:1002FE00700375A300AE5CAF5D74066F4E70037530
:10030E00A300AE5CAF5D74076F4E700375A300AEB5
:10031E005CAF5D74086F4E700375A300AE5CAF5D8D
:10032E007408BE00039F5016AC5AAD5BED2FFFEC68
:10033E003EFE90007012662DE5A3F075A300AE5C34
:10034E00AF5DEFB41009EEB4010574141265E6AE9C
:10035E005CAF5DEFB41007EEB4010375F80D785C79
:10036E0012665A02029722755D00755C0075F809D7
:10037E00AE5CAF5D7417BE0004D39F500302044DF4
:10038E00A2F9B3500302044AE55D455C700375A300
:10039E00D2AE5CAF5D74016F4E700375A300AE5CA0
:1003AE00AF5D74026F4E700D9007BAE075F002A447
:1003BE00FDACF08DA3AE5CAF5D74036F4E70037534
:1003CE00A300AE5CAF5D74046F4E700375A300AEF8
:1003DE005CAF5D74056F4E700375A300AE5CAF5DD0
:1003EE0074066F4E700375A300AE5CAF5D74076F3D
:1003FE004E700375A300AE5CAF5D74086F4E700354
:10040E0075A300AE5CAF5D7408BE00039F500C90E8
:10041E00005212662DE5A3F075A300AE5CAF5D74BD
:10042E00166F4E700574141265E6AE5CAF5D7416F1
:10043E006F4E700375F80D785C12665A02037E22B9
:10044E00900045E0B4AB0280030204E8755D0075D0
:10045E005C0075F809AE5CAF5D7412BE007CD39F74
:10046E004078A2F9B34070E55D455C700375A382D8
:10047E00AE5CAF5D74016F4E700375A300AE5CAFE2
:10048E005D74026F4E700D9007BAE075F002A4FD18
:10049E00ACF08DA3AE5CAF5D74036F4E700375A3AD
:1004AE0000AE5CAF5D7403BE00039F500990005711
:1004BE0012662DE0F5A3AE5CAF5D74116F4E700544
:1004CE0074141265E6AE5CAF5D74116F4E700375F9
:1004DE00F80D785C12665A020463229007C8E4F0A5
:1004EE0074649007B9F8E4F0E8A3F012037574C8C9
:1004FE009007B9F8E4F0E8A3F074FF900052F0749E
:10050E00FF900053F074FF900054F0740090004C74
:10051E00F074FF900055F07400900057F074019045
:10052E000058F090005EE0B4371A90005BE0900047
:10053E0052F090005CE0900053F090005DE090006F
:10054E0054F080469007C87401F074659007B9F8AE
:10055E00E4F0E8A3F012037574C89007B9F8E4F05C
:10056E00E8A3F090005EE0B4371A90005BE09000D4
:10057E0052F090005CE0900053F090005DE090002F
:10058E0054F0800674029007C8F09007C9E4F07426
:10059E00669007B9F8E4F0E8A3F012037574C890FA
:1005AE0007B9F8E4F0E8A3F090005DE0B4371290DC
:1005BE00005BE090004CF090005CE0900055F08005
:1005CE00769007C97401F074679007B9F8E4F0E803
:1005DE00A3F012037574C89007B9F8E4F0E8A3F01D
:1005EE0090005DE0B4371290005BE090004CF0900C
:1005FE00005CE0900055F0803E74029007C9F074E4
:10060E00689007B9F8E4F0E8A3F012037574C89087
:10061E0007B9F8E4F0E8A3F090005DE0B43712906B
:10062E00005BE090004CF090005CE0900055F08094
:10063E000674039007C9F022E54E64046006E5993E
:10064E0064FF60028031A23A4004D23A8027E54E20
:10065E00600874E6254E900048F0E54D600874F091
:10066E00254D900048F0E54EB4010280FE754E0017
:10067E00754D00C23A8002C23AE54E90384AF828CB
:10068E002873754E00E599B4FF03754D01E599B4D5
:10069E00FE03754D02E599B4FD03754D03E599B45E
:1006AE00FC03754D04E599B4FA03754D05E599B44F
:1006BE00FB06754E01124022E599B4F906754E04FB
:1006CE00124022E599D394E54007E599C394F04092
:1006DE0002801685994F754E027E017F00E54FC34D
:1006EE0094E61266068E328F339007BDE4F0A3F0C7
:1006FE00E599D394C44007E599C394E64002802857
:10070E0085994F754E0374E5C3954FF533753200D9
:10071E00AE32AF33905EDE1265D5E493F87401937A
:10072E009007BDC8F0A3C8F0D299020C5690005B9A
:10073E00E07005A22CB3400280429007BDE0FEA3FC
:10074E00E0FF74FFBE00039F5009EFC39446EE9482
:10075E000640119007BDE0FEA3E0FFEFD3946DEECF
:10076E00940640139007BDE0FEA3E0FF90007912BF
:10077E00662DE599F0800385997480119007BDE090
:10078E00FEA3E0FF90007912662DE599F09007BD6B
:10079E001266149007BDE0FEA3E0FFEFB40106EE73
:1007AE00B4070280030209FD900779E0B43C028091
:1007BE00030209FDA22C50030208E8C29C90005BC4
:1007CE00E0900117F090005CE0900086F090005DE4
:1007DE00E09000A6F090005EE09000CFF090005FF9
:1007EE00E090007BF0900060E09000C1F09000611E
:1007FE00E09000DFF0900062E09000B3F0900063B4
:10080E00E09000D1F0900064E0900101F09000655E
:10081E00E0900165F0900066E0900166F090006750
:10082E00E0900167F0123B9490006DE09000E8F0CC
:10083E0090006EE090009FF090006FE09000A0F0AE
:10084E0074639007B9F8E4F0E8A3F074AB90004538
:10085E00F012044E900045E4F07464F5097508003A
:10086E001200E9A2214039757301E573D394075044
:10087E002DE5739007B9F8E4F0E8A3F074AA9000A0
:10088E0045F0120115E573C39407500A7464F50917
:10089E007508001200E97873740126F650CC803783
:1008AE00757308E573D3940E502DE5739007B9F860
:1008BE00E4F0E8A3F074AA900045F0120115E57378
:1008CE00C3940E500A7464F5097508001200E97895
:1008DE0073740126F650CC0209E7C29C900117E012
:1008EE0090005BF0900086E090005CF09000A6E037
:1008FE0090005DF09000CFE090005EF090007BE005
:10090E0090005FF09000C1E0900060F09000DFE09A
:10091E00900061F09000B3E0900062F09000D1E0A2
:10092E00900063F0900101E0900064F0740090007C
:10093E0065F07400900066F07400900067F07463C8
:10094E009007B9F8E4F0E8A3F074AB900045F0120C
:10095E00044E900045E4F07464F509750800120029
:10096E00E9757301E573D394075026E5739007B9C3
:10097E00F8E4F0E8A3F074AA900045F012011574A3
:10098E0064F5097508001200E97873740126F650B3
:10099E00D3D29C7599FB743C900779F0757308E57A
:1009AE0073D3940E5026E5739007B9F8E4F0E8A3DC
:1009BE00F074AA900045F01201157464F5097508DB
:1009CE00001200E97873740126F650D374C89007AC
:1009DE00B9F8E4F0E8A3F080FE74C89007B9F8E423
:1009EE00F0E8A3F0D29C754E00754D007599FB0290
:1009FE000C569007BDE0FEA3E0FFEF4E7006859902
:100A0E00317530009007BDE0FEA3E0FF74016F4E1C
:100A1E00701BAC30AD31AA32AB33ED2BFBEC3AFA96
:100A2E008A068B0790007912662DE599F09007BD26
:100A3E001266149007BDE0FEA3E0FF74026F4E70C5
:100A4E0021AC30AD3174566D4C7006E54F64E660E6
:100A5E00028003124022123B94854F99754E007509
:100A6E004D00020C569007BDE0FEA3E0FF9000790A
:100A7E0012662DE599F09007BD1266149007BDE041
:100A8E00FEA3E0FFAC32AD338F028E038C068D07D2
:100A9E00905F221265D5E493F9740193FEEAD39E1A
:100AAE00EB994009854F99754E00754D00020C5615
:100ABE009007BDE0FEA3E0FF90007912662DE59948
:100ACE00F09007BD1266149007BDE0FEA3E0FFEFA5
:100ADE00B40006EEB401028003020C56900054E0FE
:100AEE00D394C7400B900054E0C394C8F550801ABD
:100AFE00900054E0D39463400B900054E0C3946490
:100B0E00F5508006900054E0F550E55075F002A4C3
:100B1E00FFAEF08F73EF900079126638EFFCE0FDB8
:100B2E00EC90007C126638EDFCE0FDEC2DB5500229
:100B3E008003020C470FEF900079126638E573FFC1
:100B4E00E0FCEF90007D126638ECFFE0FCEFC39CFA
:100B5E00B550028003020C47E57390007B12663895
:100B6E00E573FFE0FCEF90007E126638ECFFE0FCD0
:100B7E00EF2CB550028003020C47E57390007F12F4
:100B8E006638E0C3955090005BF0E57390008012DC
:100B9E006638E0C3955090005CF0E57390008112CA
:100BAE006638E0C3955090005DF0740090005EF0E2
:100BBE0074FF90005FF0E573900083126638E0C317
:100BCE009550900060F0E573900084126638E0C393
:100BDE009550900061F0E573900085126638E0C381
:100BEE009550900062F0E573900082126638E0C373
:100BFE0095509007B9F8E4F0E8A3F074AB90004577
:100C0E00F012044E7464F5097508001200E990079D
:100C1E00B912661412044E7464F5097508001200B8
:100C2E00E99007B912661412044E7599F97464F5B9
:100C3E00097508001200E980FE7599FF7464F509C4
:080C4E007508001200E980FEA8
:0F384A0002069002073B020A00020A73020ABE3E
:100C560022E54D903859F8282873020D699007BD92
:100C6600E0FEA3E0FF90004A12662DE0F59990079A
:100C7600BD1266149007BDE0FEA3E0FF74116F4E2F
:100C86007003754D00020D69856E99020D69900716
:100C9600BDE0FEA3E0FF90007912662DE0F599EF26
:100CA600B40107EEB40703754D009007BD12661434
:070CB600020D699007BEE08A
:0F385900020C60020C63020C8E020C94020CB97C
:100CBD00903A0CF8282873855399020D5E855F993B
:100CCD00020D5E856199020D5E856599020D5E8549
:100CDD006799807D85689980788569998073856A23
:100CED0099806E90001AE0F5998066A23BB340079B
:100CFD007599FAC23B8041A22BB3400575990F80BF
:100D0D00359007C8E0600A9007C8E024DCF59980AB
:100D1D00169007C9E0600A9007C9E024DEF59980B6
:100D2D0006900048E0F599900048E4F09007C8E47B
:100D3D00F09007C9E4F0C22B8017856B998012855E
:100D4D006699800D856C9980087599FC8003754DA9
:010D5D000095
:103A0C00020CC4020CCA020CD0020CD6020CDC0252
:103A1C000CE1020CE6020CEB020CF0020CF8020DAD
:0D3A2C0047020D4C020D51020D56020D5BBC
:0B0D5E009007BD1266148003123A39A2
:03386800020D66E8
:100D690022E537255BFFAE5A50010E9000791266D5
:100D79002DE0F538E537255BFFAE5A50010E0FBF60
:100D890000010E90007912662DE0F539853F3BE5AB
:100D990038B539058538378041E539D39538401D4F
:100DA900E539C39538853AF0A4FFAEF0E53B8E04EA
:100DB9008F05FF1265F6ED2538F537801DE538C337
:100DC9009539853AF0A4FFAEF0E53B8E048F05FF17
:100DD9001265F6EDF4042538F53722E539D395384F
:100DE900401DE539C39538853AF0A4FFAEF0E53BDF
:100DF9008E048F05FF1265F6ED2538F537801DE560
:100E090038C39539853AF0A4FFAEF0E53B8E048FDF
:100E190005FF1265F6EDF4042538F5372290007FB9
:100E2900E0B40170E56775F00A84FF7E008F37E54D
:100E39006775F00A84ADF07C008D3A753F0A755AE2
:100E490005755B24E537C394115005120D6A8006B8
:100E59009005AEE0F537E537900072F0E56775F07B
:100E69000A84FF7E008F37E56775F00A84ADF07C50
:100E7900008D3A753F0A755A05755B5AE537C39473
:100E8900115005120D6A80069005E4E0F537E53743
:100E9900900012F02290007FE0B4016AE56775F0D6
:100EA9000A84FF7E008F37E56775F00A84ADF07C10
:100EB900008D3A753F0A755A05755B36E537C39457
:100EC900115005120D6A80069005C0E0F537853787
:100ED9004BE56775F00A84FF7E008F37E56775F08B
:100EE9000A84ADF07C008D3A753F0A755A05755B29
:100EF90048E537C394115005120D6A80069005D252
:100F0900E0F53785374C22E55F75F00484FF7E00F4
:100F19008F37E55F75F00484ADF07C008D3A753F3D
:100F290004755A01755B00E537C3943F5005120DEE
:100F39006A80069001B8E0F5378537297528009051
:100F49000047E075F020A4FFAEF09000CAE08E04DF
:100F59008F05FF1265F68D379000B2E0D3955F508B
:100F6900030210169000D6E0D3955F4010ED900172
:100F7900B9126638E0F52B752A000210139000A10A
:100F8900E0D3955F4043E5379001B9126638E0F543
:100F990038E5379001D9126638E0F5399000D6E086
:100FA900F404255FF53A9000A1E0FE9000D6E0F444
:100FB900042EF53BE538B539058538378003120D20
:100FC900E485372B752A008041E5379001D91266EF
:100FD90038E0F538E5379001F9126638E0F53990CF
:100FE90000A1E0F404255FF53A9000B2E0FE90001C
:100FF900A1E0F4042EF53BE538B53905853837808D
:1010090003120DE485372B752A000210BD9000D913
:10101900E0D3955F5011E537900239126638E0F553
:101029002B752A000210BD9000A2E0D3955F5043B2
:10103900E537900219126638E0F538E5379002393C
:10104900126638E0F5399000A2E0F404255FF53A1C
:101059009000D9E0FE9000A2E0F4042EF53BE538BB
:10106900B539058538378003120DE485372B752A84
:10107900008041E5379001F9126638E0F538E53727
:10108900900219126638E0F5399000B2E0F40425AF
:101099005FF53A9000A2E0FE9000B2E0F4042EF56C
:1010A9003BE538B539058538378003120DE48537B6
:1010B9002B752A00229000EAE0F53C753F11755A1C
:1010C90002755B00AE52AF53E53C75F00FA4FDAC61
:1010D900F0EDD39FEC9E4021E53C8E048F05FF1275
:1010E90065F6ED75F010A4FFAEF0E55F75F01184BB
:1010F900FD7C00ED2FF53D800EE55F75F01184FF55
:101109007E00EF24F0F53D853D37E55F75F01184EC
:10111900AFF07E008F3A120D6A85373EAE52AF535B
:101129009000EAE075F00FA4FDACF0EDD39FEC9EC2
:101139004028755A02755B10853D37120D6A853E48
:1011490038853739AE52AF53E53C8E048F05FF120F
:1011590066218D3A853C3B120DE4853729752800B7
:10116900752B64752A00229000EAE0F53C753F1161
:10117900755A02755B00AE52AF53E53C75F00FA48A
:10118900FDACF0EDD39FEC9E4021E53C8E048F052C
:10119900FF1265F6ED75F010A4FFAEF0E56175F08C
:1011A9001184FD7C00ED2FF53D800EE56175F01190
:1011B90084FF7E00EF24F0F53D853D37E56175F04C
:1011C9001184AFF07E008F3A120D6A85373EAE5218
:1011D900AF539000EAE075F00FA4FDACF0EDD39F9A
:1011E900EC9E4028755A02755B10853D37120D6AD1
:1011F900853E38853739AE52AF53E53C8E048F05AD
:10120900FF1266218D3A853C3B120DE4853729751D
:101219002800E56B6017E56BC394FE50109000DE63
:10122900E0B402099000CCE0D3940B50028017AED1
:1012390028AF29E56B12660674E78E048F05FF1245
:1012490065F68C288D299000B4E0B40453E55F75E8
:10125900F00484FF7E008F37E55F75F00484ADF0FC
:101269007C008D3A753F04755A01755B00E537C3FB
:10127900943F5005120D6A80069001B8E0F537AE2B
:1012890028AF29E53712660674648E048F05FF12AC
:1012990065F6AE28AF29EF2DFDEE3CFC8C288D2993
:1012A900752B64752A002290007FE0B40146E5673A
:1012B90075F00A84FF7E008F37E56775F00A84AD03
:1012C900F07C008D3A753F0A755A05755B00E53764
:1012D900C394115005120D6A800690058AE0F5370E
:1012E900AE2AAF2BE5372FFF50010E746412664A00
:1012F9008E2A8F2B900080E0B40146E56875F00ACC
:1013090084FF7E008F37E56875F00A84ADF07C00B4
:101319008D3A753F0A755A05755B6CE537C39411AB
:101329005005120D6A80069005F6E0F537AE2AAF32
:101339002BE5372FFF50010E746412664A8E2A8FEF
:101349002B90008FE0B40249E56AC3944175F0051A
:1013590084FF7E008F37E56A75F00584ADF07C0067
:101369008D3A753F05755A06755B00E537C39413C9
:101379005005120D6A800690068CE0F537AE2AAF4B
:101389002BE5372FFF50010E746412664A8E2A8F9F
:101399002B9000D1E0B40202800302144FE55F757F
:1013A900F01584FF7E008F37E55F75F01584ADF089
:1013B9007C008D3A753F15755A03755BF4E537C3A3
:1013C900940B5005120D6A8006900478E0F537E514
:1013D9003775F0FFA4FFAEF09000D2E08E048F05C0
:1013E900FF1265F6ED90006BF0E56675F078A4FFE5
:1013F900AEF074FF8E048F05FF1265F68C5A8D5B73
:1014090074028C068D071200398F37AC5AAD5B74A4
:1014190004FF1266218D3A753F04755A06755B28DB
:10142900E537C3941D5005120D6A80069006BEE08B
:10143900F537AE2AAF2BE5372FFF50010E74641232
:10144900664A8E2A8F2B90007EE0B4025DE56175B5
:10145900F064A4FFAEF074081200398E5C8F5D74DD
:10146900058E048F05FF1265F68D37AE5CAF5D748E
:10147900058E048F05FF1266218D3A753F05755A51
:1014890005755BDEE537C394135005120D6A8006B6
:1014990090066AE0F537AE2AAF2BE5372FFF5001EA
:1014A9000E746412664A8E2A8F2B9000C0E0703C3D
:1014B900900047E075F00584FF7E008F3790004764
:1014C900E075F00584ADF07C008D3A753F05755ADD
:1014D90005755BC0E537C3941D5005120D6A80067A
:1014E900900656E0F537E537900073F022900087B3
:1014F900E0B401179007C4E0252BFFAE2A50010E76
:101509009000DBE012664A8E2A8F2B9000FFE0B430
:101519000114900100E0A852B8000495535007E562
:101529005FC39560400280129000A9E0252BFFAEB1
:101539002A50010E8E2A8F2B802F900087E0B4034A
:1015490016A22EB3B350109007C7E0C39405A85252
:10155900B800069553400280109000A9E0252BFFA2
:10156900AE2A50010E8E2A8F2B900081E0B4020220
:1015790080030218F4900084E0602FE567D3944655
:101589004028900013E0FEA3E0FF9000BFE075F053
:1015990003A4FDACF0EFD39DEE9C400E9000E3E078
:1015A900A852B80005D3955350030218F49000B41B
:1015B900E0B40302800302175885615B755A0090F5
:1015C900008BE0A852B800049553500E90008CE0AF
:1015D900A85AB80005D3955B5003021755E5617504
:1015E900F002A4FFAEF074158E048F05FF1265F6A4
:1015F9008C068D0790060912662DFEE0FFEE90001D
:1016090083E0FEEF8E0088F0A4FFAEF074648E04D0
:101619008F05FF1265F68C5A8D5B900047E075F0D7
:1016290018A4FFAEF09000CAE08E048F05FF126582
:10163900F68C068D0790062112662DAE5AAF5BE037
:1016490012660674648E048F05FF1265F68C5A8D36
:101659005BE565A85AB80077D3955B4072E565C329
:10166900955BFFE4955AFE8E5A8F5B7428BE000382
:101679009F500C755B28755A00740D900048F0AEA8
:101689005AAF5B900084E012660674288E048F05B9
:10169900FF1265F68C5A8D5BAE28AF29740A8E0449
:1016A9008F05FF1265F68D068C07AC5AAD5BCFCE60
:1016B900CF120003740A8E048F05FF1265F68C5A47
:1016C9008D5BAE28AF291266528E288F29807DE561
:1016D90065A85AB80004955B5072AE5AAF5BE565D0
:1016E90012664A8E5A8F5B7428BE00039F500C7590
:1016F9005B28755A00740D900048F0AE5AAF5B90A4
:101709000084E012660674288E048F05FF1265F6C0
:101719008C5A8D5BAE28AF29740A8E048F05FF128F
:1017290065F68D068C07AC5AAD5BCFCECF120003A0
:10173900740A8E048F05FF1265F68C5A8D5BAE28EC
:10174900AF29EF2DFDEE3CFC8C288D290218F49071
:1017590000CCE0855FF0A4FFAEF074051266067454
:10176900071200398E5A8F5B90008BE0A852B8009F
:10177900049553501290008CE075F002A4FDACF072
:10178900EFC39DEE9C40030218F4E55F75F00B84EE
:10179900FF7E0090060912662DFEE0FFEE900083A1
:1017A900E0FEEF8E0088F0A4FFAEF074648E048F23
:1017B90005FF1265F68C5A8D5B900047E075F018AD
:1017C900A4FFAEF09000CAE08E048F05FF1265F603
:1017D9008C068D0790062112662DAE5AAF5BE0127A
:1017E900660674648E048F05FF1265F68C5A8D5B4C
:1017F900E565A85AB80077D3955B4072E565C3954E
:101809005BFFE4955AFE8E5A8F5B7428BE00039FD6
:10181900500C755B28755A00740D900048F0AE5A4B
:10182900AF5B900084E012660674288E048F05FF72
:101839001265F68C5A8D5BAE28AF29740A8E048F17
:1018490005FF1265F68D068C07AC5AAD5BCFCECF7E
:10185900120003740A8E048F05FF1265F68C5A8DE7
:101869005BAE28AF291266528E288F29807DE565E7
:10187900A85AB80004955B5072AE5AAF5BE5651281
:10188900664A8E5A8F5B7428BE00039F500C755BA5
:1018990028755A00740D900048F0AE5AAF5B90005D
:1018A90084E012660674288E048F05FF1265F68C93
:1018B9005A8D5BAE28AF29740A8E048F05FF126515
:1018C900F68D068C07AC5AAD5BCFCECF12000374F0
:1018D9000A8E048F05FF1265F68C5A8D5BAE28AF10
:1018E90029EF2DFDEE3CFC8C288D29229000DFE0AC
:1018F900B4026AE55F75F00884FF7E008F37E55F03
:1019090075F00884ADF07C008D3A753F08755A0171
:10191900755BE0E537C3943F5005120D6A80069068
:101929000278E0F53785372D752C00AE2CAF2DAC3C
:101939002AAD2B12000374648E048F05FF1265F61D
:101949008C2C8D2D90007CE08C068D071266067418
:10195900648E048F05FF1265F68C2C8D2DAE28AF91
:1019690029AC2AAD2B12000374648E048F05FF1273
:1019790065F68C288D2990007CE08C068D0712660F
:101989000674648E048F05FF1265F68C288D29A2D2
:101999000D401DAE52AF537405BE00039F5002D2D5
:1019A9000DE561D394CC4008D2017411900048F040
:1019B9009000DEE0B402089000CCE0640B60028085
:1019C90035AE28AF29E56B12660674E78E048F05DC
:1019D900FF1265F68C288D299000DFE0B40217AE5E
:1019E9002CAF2DE56B12660674E78E048F05FF1286
:1019F90065F68C2C8D2D90009EE05402601B9000A2
:101A090095E0A852B80012D39553400DA20DB3B377
:101A19005007E561C3949A40028028AE34AF3590EF
:101A29000093E075F002A4FDACF0EF2DFDEE3CFC57
:101A390074022DFD50010CE561BC0007D39D4003E4
:101A4900754301856135753400E5437003021B3820
:101A59009000F1E0C395435003021B2A900101E075
:101A6900C394025076E56775F00A84FF7E009005FD
:101A79007912662DE0F55B755A00AE5AAF5B90009E
:101A890094E012660674648E048F05FF1265F68C65
:101A99005C8D5D9000F1E004C395438C068D0712BF
:101AA90066069000F1E08E048F05FF1265F68C5CE6
:101AB9008D5DAE28AF29EF2DFDEE3CFC8C288D29DC
:101AC9009000DFE0B40212AE2CAF2DAA5CAB5DEF43
:101AD9002BFBEE3AFA8A2C8B2D80469000F1E0041C
:101AE900C39543854BF0A4FFAEF09000F1E08E045E
:101AF9008F05FF1265F68C5C8D5DAE28AF29EF2D41
:101B0900FDEE3CFC8C288D299000DFE0B40212AE7A
:101B19002CAF2DAA5CAB5DEF2BFBEE3AFA8A2C8B2E
:101B29002D05439000F1E0C39543500375430090A0
:101B3900009EE05401601B900092E0A852B8001288
:101B4900D39553400DA20DB3B35007E55FC394CCB1
:101B590040028025900090E075F003A4FFAEF0E507
:101B6900402FFF50010E74032FFF50010EE55FBE99
:101B79000007D39F4003754401855F40E544700326
:101B8900021C6B9000F2E0C395445003021C5D9067
:101B99000101E0C394025076E56775F00A84FF7E7F
:101BA9000090057912662DE0F55B755A00AE5AAFC3
:101BB9005B900091E012660674648E048F05FF1233
:101BC90065F68C5C8D5D9000F2E004C395448C064B
:101BD9008D071266069000F2E08E048F05FF1265EC
:101BE900F68C5C8D5DAE28AF29EF2DFDEE3CFC8CAB
:101BF900288D299000DFE0B40212AE2CAF2DAA5C2B
:101C0900AB5DEF2BFBEE3AFA8A2C8B2D80469000C8
:101C1900F2E004C39544854CF0A4FFAEF09000F2C5
:101C2900E08E048F05FF1265F68C5C8D5DAE28AFE2
:101C390029EF2DFDEE3CFC8C288D299000DFE0B4C6
:101C49000212AE2CAF2DAA5CAB5DEF2BFBEE3AFA7C
:101C59008A2C8B2D05449000F2E0C39544500375FE
:101C690044009000F4E02529FFAE2850010E8E288B
:101C79008F299000A3E0A828B8000495295009905D
:101C890000A3E0F5297528009000DFE0B4020D906B
:101C990000A3E0A82CB80006952D40028009900009
:101CA900A3E0F52D752C00229000DFE0B40102803D
:101CB90003021DBCA20DB35003021DBA9000AAE095
:101CC900B40168AE28AF29AC52AD53120003743C7D
:101CD9008E048F05FF1265F69000BAE0BC00109DD6
:101CE900400D9000BCE0A828B8000495295002D204
:101CF90002AE28AF29AC52AD53120003743C8E04D6
:101D09008F05FF1265F69000BAE0C3940ABC00156E
:101D1900D39D40119000BCE0C39405A828B80005E4
:101D2900D3952950028002C2028068AE28AF29AC3F
:101D390052AD5312000374788E048F05FF1265F6B5
:101D49009000BAE0BC00109D400D9000BCE0A828AE
:101D5900B8000495295004D2028038AE28AF29ACC6
:101D690052AD5312000374788E048F05FF1265F685
:101D79009000BAE0C3940ABC0015D39D40119000AD
:101D8900BCE0C39405A828B80005D3952950028062
:101D990002C202A202B34019AE28AF299000BBE0EB
:101DA90012660674648E048F05FF1265F68C288D01
:101DB900298002C202A200B34006A201B3B35009AE
:101DC900900019E4F0A3F08024AE28AF297400D361
:101DD9009F74019E400C900019E528F0A3E529F0B5
:101DE900800B74FF900019F8E4F0E8A3F09000C1AB
:101DF900E0D39402400C9000ACE07006A20DB3B39E
:101E09004002801AAE28AF2974021266068E288F06
:101E190029AE2CAF2D74021266068E2C8F2D9000E0
:101E2900AAE0B4011AAE28AF2974021266068E28F8
:101E39008F29AE2CAF2D74021266068E2C8F2DAE13
:101E490028AF29745E126606740A8E048F05FF1284
:101E590065F68C288D299000DFE0B40217AE2CAF0F
:101E69002D745E126606740A8E048F05FF1265F6DC
:101E79008C2C8D2DAE28AF297402BE000AD39F4049
:101E890006752902752800AE2CAF2D7402BE000A12
:101E9900D39F4006752D02752C00900017E528F098
:101EA900A3E529F022900047E0900379126638E013
:101EB900F541754264900047E0FE9000B5E0D39E7D
:101EC9004037E55F75F00884FF7E008F37E55F7561
:101ED900F00884ADF07C008D3A753F08755A03759A
:101EE9005B96E537C3941F5005120D6A800690046E
:101EF9002EE0F5378537428035E55F75F00884FFB8
:101F09007E008F37E55F75F00884ADF07C008D3A6F
:101F1900753F08755A03755BB6E537C3941F5005BD
:101F2900120D6A800690044EE0F5378537422290FB
:101F390000EBE0F53C753F11755A04755B00AE5234
:101F4900AF53E53C75F00FA4FDACF0EDD39FEC9ECB
:101F59004021E53C8E048F05FF1265F6ED75F01002
:101F6900A4FFAEF0E55F75F01184FD7C00ED2FF55F
:101F79003D800EE55F75F01184FF7E00EF24F0F5DA
:101F89003D853D37E55F75F01184AFF07E008F3AEE
:101F9900120D6A85373EAE52AF539000EBE075F0F3
:101FA9000FA4FDACF0EDD39FEC9E4028755A047543
:101FB9005B10853D37120D6A853E38853739AE523B
:101FC900AF53E53C8E048F05FF1266218D3A853C9F
:101FD9003B120DE4853741754264229000EBE0F530
:101FE9003C753F11755A04755B00AE52AF53E53C21
:101FF90075F00FA4FDACF0EDD39FEC9E4021E53CBC
:102009008E048F05FF1265F6ED75F010A4FFAEF092
:10201900E56175F01184FD7C00ED2FF53D800EE53D
:102029006175F01184FF7E00EF24F0F53D853D37A1
:10203900E56175F01184AFF07E008F3A120D6A8563
:10204900373EAE52AF539000EBE075F00FA4FDACF4
:10205900F0EDD39FEC9E4028755A04755B10853DC1
:1020690037120D6A853E38853739AE52AF53E53C94
:102079008E048F05FF1266218D3A853C3B120DE4D3
:102089008537417542649000B4E0B4047990004703
:10209900E0FE9000B5E0D39E4037E55F75F0088417
:1020A900FF7E008F37E55F75F00884ADF07C008D09
:1020B9003A753F08755A03755B96E537C3941F5007
:1020C90005120D6A800690042EE0F53785374280A7
:1020D90035E55F75F00884FF7E008F37E55F75F0A1
:1020E9000884ADF07C008D3A753F08755A03755B1D
:1020F900B6E537C3941F5005120D6A800690044E49
:10210900E0F5378537422290007FE0B4013BE5676F
:1021190075F00A84FF7E008F37E56775F00A84AD94
:10212900F07C008D3A753F0A755A05755B12E537E3
:10213900C394115005120D6A800690059CE0F5378D
:10214900E5422537C39464F542900080E0B4013B31
:10215900E56875F00A84FF7E008F37E56875F00A37
:1021690084ADF07C008D3A753F0A755A05755B7E22
:10217900E537C394115005120D6A8006900608E0F0
:10218900F537E5422537C39464F542E5412542F523
:1021990036900087E0B402109007C3E02536FE9020
:1021A90000DBE0F4042EF5369000DEE0D394014024
:1021B90040E56BC394E7501D74E7C3956BFE900728
:1021C900C5E08E00F5F0E884FF7E008F37E53625FF
:1021D90037F536801CE56BC394E7FE9007C5E08EA2
:1021E90000F5F0E884FF7E008F37E536C39537F5B3
:1021F90036A20D4006E5412464F536E536D39464EC
:102209004009E536C39464F53680037536009000BD
:10221900B7E0C3953650069000B7E0F53622D200F4
:10222900900071E0A852B800049553504190007194
:10223900E0A852B800049553500375360F90007109
:10224900E004A852B800049553500375360A90006B
:1022590071E02402A852B80004955350057536055B
:10226900C200900071E060067409900048F0C23E17
:102279007E017F009000BDE01266069000CCE08EE2
:10228900048F05FF1265F6E55FBC0017D39D401367
:102299009000C6E0B40204D23E8002C200740A90E3
:1022A9000048F09000BEE0C3956750159000D0E05B
:1022B900A852B8000495535002C200740B9000480C
:1022C900F0E567C39464501D900116E0600D90011C
:1022D90016E0A852B80006955340028008C200745F
:1022E9000B900048F0A20040037536059000FFE00E
:1022F900B40114900100E0A852B8000495535007A6
:10230900E55FC39560400280089000A8E0F536803B
:102319003A900087E0B40306A22EB3B34002802BA3
:102329009007C7E0C39405A852B800049553500C10
:102339009000A8E0F536740C900048F09007C7E0CB
:10234900A852B8000495535002C20085366C90001B
:1023590079E02536FE900047E075F01E84FC7F0089
:10236900EE2CF53622900047E075F00584FF7E00DB
:102379008F37900047E075F00584ADF07C008D3A09
:10238900753F05755A03755BD69000CAE01475F060
:102399000584FF7E00E537BE00039F5005120D6AD4
:1023A900800BE53790044F126638E0F537E5379032
:1023B90007C6F09007C6E0FE9000B9E0C39E50083A
:1023C9009000B9E09007C6F022E56775F00A84FF2E
:1023D9007E0090057912662DE0F546E546D39464B2
:1023E9004010E546C3946475F00F84FF7E008F4664
:1023F900800375460090009CE02546F54622900032
:10240900B4E0C3940350269007B3E0FEA3E0FF7441
:1024190004120039E55F126606740F8E048F05FFFA
:102429001265F69007B1ECF0A3EDF080249007B3A4
:10243900E0FEA3E0FF7404120039E5611266067438
:102449000F8E048F05FF1265F69007B1ECF0A3ED2E
:10245900F090008FE0B40262E56AC3944175F0051B
:1024690084FF7E008F37E56A75F00584ADF07C0046
:102479008D3A753F05755A06755B14E537C3941790
:102489005005120D6A80069006A0E0F5379007B155
:10249900E0FEA3E0FF740A8E048F05FF1265F6E5DE
:1024A900378C068D07126606740A8E048F05FF1293
:1024B90065F69007B1ECF0A3EDF09007B1E0FEA34B
:1024C900E0FF9007B7E0FCA3E0FDEDD39FEC9E4051
:1024D9000F9007B7E0F8A3E09007B1C8F0A3C8F0E0
:1024E900229006C0E090386BF8282873804C8553F9
:1024F9007380479000CCE0855FF0A4FFAEF07408CC
:102509001200398F738033856173802E85677380DC
:10251900298568738024856973801F856A73801A89
:10252900856B7380158566738010856573800B854F
:0A2539006C73800690001AE0F57341
:10386B000224F50224F70224FC022510022515027E
:10387B00251A02251F02252402252902252E0225A1
:07388B003302253802253D40
:102543009006C1E0FE9006C2E0D39E404B9006C0C9
:10255300E0B404189006C2E0C395735002D22F90E2
:1025630006C1E0D395734002C22F802A9006C1E0D2
:10257300C3957350099006C2E0D39573500280024D
:10258300D22F9006C1E0D3957350099006C2E0C3E1
:1025930095735002C22F802A9006C1E0D3957340F1
:1025A300099006C2E0C3957340028002C22F9006D1
:1025B300C1E0C3957340099006C2E0D3957340020E
:1025C300D22F229006C4E0903892F8282873804CCA
:1025D30085537380479000CCE0855FF0A4FFAEF095
:1025E30074081200398F738033856173802E856779
:1025F3007380298568738024856973801F856A7356
:10260300801A856B7380158566738010856573806A
:0C2613000B856C73800690001AE0F573D4
:103892000225D10225D30225D80225EC0225F10208
:1038A20025F60225FB02260002260502260A02262A
:0738B2000F02261402261983
:10261F009006C5E0FE9006C6E0D39E405F9006C4CC
:10262F00E0B404189006C6E0C395735002D2309000
:10263F0006C5E0D395734002C230803E9006C5E0D8
:10264F00C3957350099006C6E0D39573500280026C
:10265F00D2309006C5E0D3957350099006C6E0C3FB
:10266F0095735002C2309006C4E0B401099000D8AF
:10267F00E0D3956150028002C230802A9006C5E0F7
:10268F00D3957340099006C6E0C39573400280024C
:10269F00C2309006C5E0C3957340099006C6E0D3DB
:1026AF0095734002D230229006C8E09038B9F828CE
:1026BF002873804C85537380479000CCE0855FF082
:1026CF00A4FFAEF074081200398F738033856173E5
:1026DF00802E856773802985687380248569738050
:1026EF001F856A73801A856B7380158566738010DA
:1026FF00856573800B856C73800690001AE0F57307
:1038B9000226C10226C30226C80226DC0226E1022C
:1038C90026E60226EB0226F00226F50226FA022651
:0738D900FF0227040227098A
:10270F009006C9E0FE9006CAE0D39E404B9006C8E3
:10271F00E0B404189006CAE0C395735002D231900A
:10272F0006C9E0D395734002C231802A9006C9E0F2
:10273F00C3957350099006CAE0D395735002800277
:10274F00D2319006C9E0D3957350099006CAE0C301
:10275F0095735002C231802A9006C9E0D395734019
:10276F00099006CAE0C3957340028002C2319006F9
:10277F00C9E0C3957340099006CAE0D39573400230
:10278F00D231229006CCE09038E0F8282873804CA4
:10279F0085537380479000CCE0855FF0A4FFAEF0C7
:1027AF0074081200398F738033856173802E8567AB
:1027BF007380298568738024856973801F856A7388
:1027CF00801A856B7380158566738010856573809D
:0C27DF000B856C73800690001AE0F57307
:1038E00002279D02279F0227A40227B80227BD02B4
:1038F00027C20227C70227CC0227D10227D60227D8
:07390000DB0227E00227E5CE
:1027EB009006CDE0FE9006CEE0D39E404B9006CCFB
:1027FB00E0B404189006CEE0C395735002D2329029
:10280B0006CDE0D395734002C232802A9006CDE00C
:10281B00C3957350099006CEE0D395735002800296
:10282B00D2329006CDE0D3957350099006CEE0C31B
:10283B0095735002C232802A9006CDE0D395734037
:10284B00099006CEE0C3957340028002C232900617
:10285B00CDE0C3957340099006CEE0D3957340024B
:10286B00D232229006D0E0903907F8282873804C9A
:10287B0085537380479000CCE0855FF0A4FFAEF0EA
:10288B0074081200398F738033856173802E8567CE
:10289B007380298568738024856973801F856A73AB
:1028AB00801A856B738015856673801085657380C0
:0C28BB000B856C73800690001AE0F5732A
:1039070002287902287B022880022894022899023B
:10391700289E0228A30228A80228AD0228B202285E
:07392700B70228BC0228C111
:1028C7009006D1E0FE9006D2E0D39E404B9006D012
:1028D700E0B404189006D2E0C395735002D2339047
:1028E70006D1E0D395734002C233802A9006D1E027
:1028F700C3957350099006D2E0D3957350028002B6
:10290700D2339006D1E0D3957350099006D2E0C335
:1029170095735002C233802A9006D1E0D395734055
:10292700099006D2E0C3957340028002C233900635
:10293700D1E0C3957340099006D2E0D39573400266
:10294700D233229006D4E090392EF8282873804C91
:1029570085537380479000CCE0855FF0A4FFAEF00D
:1029670074081200398F738033856173802E8567F1
:102977007380298568738024856973801F856A73CE
:10298700801A856B738015856673801085657380E3
:0C2997000B856C73800690001AE0F5734D
:10392E0002295502295702295C02297002297502C3
:10393E00297A02297F02298402298902298E0229E5
:07394E009302299802299D54
:1029A3009006D5E0FE9006D6E0D39E404B9006D429
:1029B300E0B404189006D6E0C395735002D2349065
:1029C30006D5E0D395734002C234802A9006D5E041
:1029D300C3957350099006D6E0D3957350028002D5
:1029E300D2349006D5E0D3957350099006D6E0C350
:1029F30095735002C234802A9006D5E0D395734074
:102A0300099006D6E0C3957340028002C234900653
:102A1300D5E0C3957340099006D6E0D39573400281
:102A2300D234229006D8E0903955F8282873804C88
:102A330085537380479000CCE0855FF0A4FFAEF030
:102A430074081200398F738033856173802E856714
:102A53007380298568738024856973801F856A73F1
:102A6300801A856B73801585667380108565738006
:0C2A73000B856C73800690001AE0F57370
:10395500022A31022A33022A38022A4C022A51024B
:103965002A56022A5B022A60022A65022A6A022A6C
:073975006F022A74022A7997
:102A7F009006D9E0FE9006DAE0D39E404B9006D840
:102A8F00E0B404189006DAE0C395735002D2359083
:102A9F0006D9E0D395734002C235802A9006D9E05B
:102AAF00C3957350099006DAE0D3957350028002F4
:102ABF00D2359006D9E0D3957350099006DAE0C36A
:102ACF0095735002C235802A9006D9E0D395734092
:102ADF00099006DAE0C3957340028002C235900672
:102AEF00D9E0C3957340099006DAE0D3957340029D
:102AFF00D235229006DCE090397CF8282873804C80
:102B0F0085537380479000CCE0855FF0A4FFAEF053
:102B1F0074081200398F738033856173802E856737
:102B2F007380298568738024856973801F856A7314
:102B3F00801A856B73801585667380108565738029
:0C2B4F000B856C73800690001AE0F57393
:10397C00022B0D022B0F022B14022B28022B2D02D3
:10398C002B32022B37022B3C022B41022B46022BF3
:07399C004B022B50022B55DA
:102B5B009006DDE0FE9006DEE0D39E404B9006DC57
:102B6B00E0B404189006DEE0C395735002D23690A1
:102B7B0006DDE0D395734002C236802A9006DDE075
:102B8B00C3957350099006DEE0D395735002800213
:102B9B00D2369006DDE0D3957350099006DEE0C384
:102BAB0095735002C236802A9006DDE0D3957340B0
:102BBB00099006DEE0C3957340028002C236900690
:102BCB00DDE0C3957340099006DEE0D395734002B8
:102BDB00D236229006E0E09039A3F8282873804C77
:102BEB0085537380479000CCE0855FF0A4FFAEF077
:102BFB0074081200398F738033856173802E85675B
:102C0B007380298568738024856973801F856A7337
:102C1B00801A856B7380158566738010856573804C
:0C2C2B000B856C73800690001AE0F573B6
:1039A300022BE9022BEB022BF0022C04022C09025E
:1039B3002C0E022C13022C18022C1D022C22022C7A
:0739C30027022C2C022C311D
:102C37009006E1E0FE9006E2E0D39E404B9006E06E
:102C4700E0B404189006E2E0C395735002D23790BF
:102C570006E1E0D395734002C237802A9006E1E08F
:102C6700C3957350099006E2E0D395735002800232
:102C7700D2379006E1E0D3957350099006E2E0C39E
:102C870095735002C237802A9006E1E0D3957340CE
:102C9700099006E2E0C3957340028002C2379006AE
:102CA700E1E0C3957340099006E2E0D395734002D3
:102CB700D237229006E4E09039CAF8282873804C6E
:102CC70085537380479000CCE0855FF0A4FFAEF09A
:102CD70074081200398F738033856173802E85677E
:102CE7007380298568738024856973801F856A735B
:102CF700801A856B73801585667380108565738070
:0C2D07000B856C73800690001AE0F573D9
:1039CA00022CC5022CC7022CCC022CE0022CE502E8
:1039DA002CEA022CEF022CF4022CF9022CFE022D06
:0739EA0003022D08022D0D60
:102D13009006E5E0FE9006E6E0D39E404B9006E485
:102D2300E0B404189006E6E0C395735002D23890DD
:102D330006E5E0D395734002C238802A9006E5E0A9
:102D4300C3957350099006E6E0D395735002800251
:102D5300D2389006E5E0D3957350099006E6E0C3B8
:102D630095735002C238802A9006E5E0D3957340EC
:102D7300099006E6E0C3957340028002C2389006CC
:102D8300E5E0C3957340099006E6E0D395734002EE
:102D9300D23822AE2EAF2F74F5D39F74019E400814
:102DA300782E12665A022EB0752F01752E00AE5280
:102DB300AF53E546BE000DD39F40099000AEE0D36C
:102DC300954740028023754700E546C39553F57345
:102DD3009000B1E0D395454008E5452573F545805E
:102DE300069000B1E0F5458002054790008AE0D3E4
:102DF3009561401CE55FC395604015AE52AF53E546
:102E030046BE00039F50099000AFE0D395484002AF
:102E1300806E9007CAE0A852B8000495535003751A
:102E23004A009007CAE0A852B8000BD39553400656
:102E3300E5539007CAF0E54A7041E553C39546F55B
:102E430073E573D3940540037573059000B0E0C335
:102E530095455007E573C3954540028009E545C391
:102E63009573F54580069000B0E0F5459000B0E01D
:102E7300D3954540069000B0E0F5457548008002C3
:102E83000548E54A701690008AE0C39561500DE548
:102E9300462405A852B8000695534002800F9000BF
:102EA3009DE0F545754A0174789007CAF022AE2E6D
:102EB300AF2F74E9D39F74039E4008782E12665A8D
:102EC30002304F752F01752E00754532A239402A05
:102ED30075451990009DE075F002A4FFAEF0E5473B
:102EE300BE0006D39F4002D2390547754A03747862
:102EF3009007CAF075490002303EAE52AF53E54623
:102F03006F4E700302303EE546BE000DD39F40096D
:102F13009000AEE0D395474002800F754700E54A25
:102F2300C394035003754519800DE546C39553F5C6
:102F330073E5472573F54790008AE0D39561400E0A
:102F43009007CAE0A852B80007D395534002800CFB
:102F5300054990009DE0B54903754A00E54AB4036D
:102F630006A20DB3B34002800A0549E549B43C0308
:102F7300754A02E54AB402299007CAE0A852B8008C
:102F83000ED395534009E5539007CAF07549009055
:102F9300008AE0C39561500975490074789007CAA7
:102FA300F0E54A705A90008AE0D39561401CE55FD2
:102FB300C395604015AE52AF53E546BE00039F5024
:102FC300099000AFE0D3954840028008754800752A
:102FD300454B8028E553C39546F573E573D39405B4
:102FE300400375730590008AE0D395614008E54876
:102FF3002573F5488006E5482406F548754900E53C
:103003004A701690008AE0C39561500DE546240589
:10301300A852B80006955340028003754A01E54A59
:10302300B40118754519054990009DE0B549067529
:103033004A0275490074789007CAF0E54575F00AAD
:10304300A4FFAEF09007BBEEF0A3EFF022E56F9084
:1030530039F1F8282873900082E0700302327790E8
:1030630000B8E0B401028003023192900046E0B55B
:103073005E02800302318F7E017F00E5BE12660689
:10308300E5BD2FFF50010E8E5A8F5B74101266063A
:10309300900070E08E048F05FF1265F69007BFEC79
:1030A300F0A3EDF074FFBC00039D500B74FF900779
:1030B300BFF8E4F0E8A3F0E56B600FE56BC394FEA3
:1030C30050089000DEE06402600280649000CCE06F
:1030D300B40B1F9007BFE0FEA3E0FF74E712660680
:1030E300E56B8E048F05FF1265F69007BFECF0A326
:1030F300EDF09000CCE0D3940B40089000B4E06472
:10310300046002802B9007BFE0FEA3E0FF9007C19D
:10311300E0FCA3E0FDEFD39DEE9C400D12665290C0
:1031230007BFEEF0A3EFF080079007BFE4F0A3F032
:10313300900082E0B4021E9007BFE0FEA3E0FF9080
:1031430007CBE02FFF50010E74011200399007BF27
:10315300EEF0A3EFF09007BFE0FEA3E0FF9007CBF4
:10316300E0BE0008D39F4004D23C8002B23C9007EB
:10317300C0E09007CBF09000B4E064016006A23C8D
:10318300B3B3400280069007C0E0F55F023275D208
:103193003C7E017F00E5BE126606E5BD2FFF5001B0
:1031A3000E8E5A8F5B7410126606900070E08E04C8
:1031B3008F05FF1265F69007BFECF0A3EDF0E56B0A
:1031C300600FE56BC394FE50089000DEE06402607C
:1031D3000280649000CCE0B40B1F9007BFE0FEA315
:1031E300E0FF74E7126606E56B8E048F05FF126538
:1031F300F69007BFECF0A3EDF09000CCE0D3940B76
:1032030040089000B4E064046002802B9007BFE0A4
:10321300FEA3E0FF9007C1E0FCA3E0FDEFD39DEE2A
:103223009C400D1266529007BFEEF0A3EFF08007AB
:103233009007BFE4F0A3F0900082E0B4021E900771
:10324300BFE0FEA3E0FF9007CBE02FFF50010E7419
:10325300011200399007BFEEF0A3EFF09007C0E032
:103263009007CBF09000B4E0640160069007C0E0E3
:10327300F55F8003755F0090007EE07006756F0157
:1032830002305075BB1802384590007EE07003028F
:1032930033FD7E017F00E5BE126606E5BD2FFF50BC
:1032A300010E8E5A8F5B9000C4E0B4010F7E0F7F36
:1032B300FFAC5AAD5B1266528E5A8F5B9000E9E009
:1032C300B40245AE5AAF5B900023E0FCA3E0FDEDF2
:1032D300D39FEC9E400A900023E55AF0A3E55BF0F0
:1032E300AE5AAF5B900025E0FCA3E0FDEFD39DEE6B
:1032F3009C400A900025E55AF0A3E55BF0AE5AAF77
:103303005B74041200398F619000E9E0704CAE5A8F
:10331300AF5B900023E0FCA3E0FDEFD39DEE9C4068
:10332300091266528E5A8F5B8006755B00755A00D0
:10333300AE5AAF5B741012660690006DE08E048F78
:1033430005FF1265F68C5A8D5B74FFBC0009D39D93
:103353004005855B6180037561FE9000B4E0B401B4
:103363000280030233FBA20DB3B3500E900088E03A
:10337300A852B80005D39553500280719000C5E060
:103383008561F0A4FFAEF074648E048F05FF1265AF
:10339300F68C5A8D5BE56B6016E56BC394FE500F9C
:1033A3009000DEE0B402089000CCE0640B60028081
:1033B30017AE5AAF5B74E7126606E56B8E048F0592
:1033C300FF1265F68C5A8D5BAE5AAF5B9007BFE078
:1033D300FCA3E0FDEDD39FEC9E4005855B5F800B76
:1033E300A23CB340069007C0E0F55F800BA23CB35C
:1033F30040069007C0E0F55F80037561009000818F
:10340300E07006756F0202305075BB1902384590A3
:103413000081E070030234B2E55ED39551400302AC
:1034230034B0900021E0FEA3E0FFE56512664A9008
:103433000021EEF0A3EFF07E017F00E5BE126606E9
:10344300E5BD2FFF50010E8E5A8F5B9000EEE070AA
:1034530013740A12660674518E048F05FF1265F603
:103463008D658019AE5AAF5B740A1266068F048E9F
:10347300057E017F95CDCCCD1264F48F65E565D3D0
:1034830094644003756564900021E0FEA3E0FFE5CA
:10349300652FFF50010E900021EEF0A3EFF0900096
:1034A30085E0048E048F05FF1265F68D6580037534
:1034B30065329000D1E07006756F0302305075BB22
:1034C300130238459000D1E0604A7E017F00E5BEDB
:1034D300126606E5BD2FFF50010E8E5A8F5B7404F2
:1034E3001200398F669000D3E08566F0A4FDACF03E
:1034F3007464FF1265F68D669000D2E08566F0A4D1
:10350300FFAEF074FF8E048F05FF1265F6ED900099
:103513006CF0800375660090007FE07006756F04A1
:1035230002305075BB1702384590007FE0B40102AA
:1035330080030235C07E017F00E5BE126606E5BD4D
:103543002FFF50010E8E5A8F5B9007CCE0601990CD
:1035530007CCE014905F6612008CE493FC74019333
:10356300FDEDC39FEC9E400280069007CCE014F073
:103573009007CCE0C394B3501DAE5AAF5B9007CC19
:10358300E004905F6612008CE493FC740193FDEFFA
:10359300C39DEE9C400280069007CCE004F09007A8
:1035A300CCE0FE9000A5E08E0088F0A4FFAEF0749E
:1035B300648E048F05FF1265F68D678003756700BF
:1035C300900080E07006756F0502305075BB1602DF
:1035D3003845900080E0B4010280030236697E0121
:1035E3007F00E5BE126606E5BD2FFF50010E8E5A21
:1035F3008F5B9007CDE060199007CDE0149060D009
:1036030012008CE493FC740193FDEDC39FEC9E4088
:103613000280069007CDE014F09007CDE0C394B389
:10362300501DAE5AAF5B9007CDE0049060D01200FE
:103633008CE493FC740193FDEFC39DEE9C400280E8
:10364300069007CDE004F09007CDE0FE9000ABE0DC
:103653008E0088F0A4FFAEF074648E048F05FF1211
:1036630065F68D68800375680075BB1F0238457E5B
:10367300017F00E5BE126606E5BD2FFF50010E8EE9
:103683005A8F5B740912660674E68E048F05FF1267
:1036930065F68D6A900087E07006756F07023050FB
:1036A30075BB15023845900087E070030237C47E6E
:1036B300017F00E5BE126606E5BD2FFF50010E8EA9
:1036C3005A8F5B74041200398F69900087E0B4014C
:1036D300159000DBE08569F0A4FFAEF074071200DB
:1036E30039EF9007C4F0900087E0B402159000DB37
:1036F300E08569F0A4FFAEF07407120039EF90077C
:10370300C3F0900087E0B4030280030237A7900060
:10371300C8E0701CE569C394195002D22EE569D341
:1037230094644002C22E9000A7E09007C7F0806324
:103733009000A7E070349000DBE08569F0A4FFAE51
:10374300F074FF8E048F05FF1265F6ED9007C7F046
:10375300AE52AF53741EBE0006D39F4002D22EE575
:1037630061D394E54002C22E8029E569C3940A50CF
:103773000DAE52AF53741EBE0004D39F500280029D
:10378300D22EE561D394E54002C22E9000A7E090CB
:1037930007C7F09007C7E0C3940550067405900768
:1037A300C7F0C23D900087E0B40414E569C39419DF
:1037B3005002D23DE569D394324002C23DC22E800D
:1037C300037569009000DEE07006756F08023050E3
:1037D30075BB14806D9000DEE060567E017F00E5CE
:1037E300BE126606E5BD2FFF50010E8E5A8F5BEFAA
:1037F300D39421EE940E4005756BFF8015AE5AAF3E
:103803005B741012660674E38E048F05FF1265F66F
:103813008D6BE56B75F00BA4FFAEF09000CCE08EE2
:10382300048F05FF1265F69007C1ECF0A3EDF0805D
:1038330003756B00900082E0600575BB1A80037509
:02384300BB18B0
:1039F10002305902328C0234120234C702352C02D1
:0B3A010035D50236720236A90237D814
:05384500056FD2EC222A
:096638002582F58250020583223F
:0F008C0025E050020583258250020583F582226C
:1065D500EF2F500205832582F582E5833E2EF58354
:0165E5002293
:10664A00CFC39FFF50011E22C3EF9DFFEE9CFE2287
:08665A000806B6000218062232
:0D661400A3E004F07006120049E004F0223B
:0E003900048007C3CE13CECF13CFD5E0F6223E
:1064F400BC000FBE0008ED8FF084FFADF022E4FE77
:10650400FF22BE000DEF60FE54F0606F20E703022F
:1065140065AAEAC0E0EBC0E078017A0075F001EE0C
:1065240020E710EF25E0FFEE33FE0AC5F023C5F0A7
:1065340030E7F0EA5407F9096A7A007B0060010841
:10654400C3EC9E40167004ED9F4010ED9FFDEC9E41
:10655400FCE5F0CA4ACA03F5F08005E5F003F5F05E
:10656400C3EE13FEEF13FFD9D77908CACBCAD8D02C
:10657400EAFEEBFFD0E0FBD0E0FA22EC8FF084FCE3
:10658400ED54F045F0C48FF084FEEDC454F045F0B2
:10659400C48FF084FDEEC4FE54F02DFFEE540F3C86
:1065A400FEADF07C0022790078008FF0EC7E0820AC
:1065B400E70DC3CD33CD33C933C9C833C8DEF08446
:1065C40049F9E5F08FF0BE00E6FD7C00E9FFE8FE46
:0165D40022A4
:0E660600F88FF0A4FFE5F0CE88F0A42EFE225F
:10000300EF8DF0A4F9A8F0EF8CF0A428F8EE8DF0B2
:06001300A428FEE9FF2213
:1065E600600D782B0265F0007830D8FED5E0F822F1
:1065F600EEC0E07E001264F4EFFDEEFCD0E0FE2279
:0C662100EEC0E07E001264F4D0E0FE2227
:03001B0002001EC2
:0300530002005652
:03009B00020071EF
:0300000002664154
:0966410075817575D00002428ECE
:0B662D00E5822FF582E5833EF5832215
:0A0049000582D5820215831582227C
:10001E00C0E0C0F0C083C082C0D075D0001241FADB
:0B002E00D0D0D082D083D0F0D0E032E0
:10005600C0E0C0F0C083C082C0D075D0001241FDA0
:10006600D0D0D082D083D0F0D0E032C0E0C0F0C093
:1000760083C082C0D075D000124219D0D0D082D0B1
:0600860083D0F0D0E0324F
:00000001FF
